:106BE200020A0A0A0A040A3204090A0A0A0A0A6496
:106BF20064645B0A640A3C0003006400050005004B
:106C02000100FF00FF0001001400C80AFF00FF009E
:106C120002000501FF01FF000100030023006300E1
:106C2200FF00FF000100FF00030006000200040055
:106C32000400FF00FF000300060AFF00FF00FF0040
:106C4200FF00FF00FF00FF00040006000600060030
:106C520006000200FF00FF00FF00FF00FF00FF0030
:106C6200FF00FF001B001B001B001B001B001B0082
:106C72001B000300030003000300030003000300E2
:106C820000000000000001000100050005000500F1
:106C920005000500050005010A00FF05FF05FF00CC
:106CA200050005000500FF00FF00FF00FF000200D5
:106CB200FF00FF00FF000100FF0005000300640069
:106CC200050005000100FF00FF0001001400C80AD2
:106CD200FF00FF0002000501FF01FF0001000300A9
:106CE2005F006300FF00FF000100FF0003000600D9
:106CF200020004000400FF00FF000300060AFF0078
:106D0200FF00FF00FF00FF00FF00FF00040006007D
:106D12000600060006000200FF00FF00FF00FF0061
:106D2200FF00FF00FF00FF001B001B001B001B00F9
:106D32001B001B001B0003000300030003000300F1
:106D42000300030000000000000001000100050034
:106D52000500050005000500050005010A00FF0504
:106D6200FF05FF00050005000500FF00FF00FF0012
:106D7200FF000200FF00FF00FF000100FF0005020C
:106D82001401000000640100003C3201000A0A0004
:106D9200030A0A0F1E00140201000101320F000053
:106DA200190000C800BE00000303030300E8030A41
:106DB20000D007B80B0302010F17181300000000E0
:106DC2000000000000000000000000000000000AB7
:106DD200050A1E0000000000000001000000000083
:106DE20001021401000000640100003C3201000AAB
:106DF2000A01030A0A4150004402010001016337FB
:106E02000000190000A8029602000303030300E831
:106E1200030A00D007B80B0302010F171813000072
:106E22000000000000000000000000000000000060
:106E3200000A280A1E0000000000000001000000F5
:106E42000000010000000000000001010909010129
:106E52001102020A0A02021204040C0C04041401B4
:106E620041CACC41D2D40041CACC41D2D40096000E
:106E720055003C002D00230019000F0005FFFBFF09
:106E8200F1FFCE0000012C0258038404B005DC0798
:106E920008083409600A8C0BB800000000000000EA
:106EA2000000000000000081F34961332505F10173
:106EB2002180F24860322404F00020C0F964705945
:106EC2005242F8405080B92430191202B8001081A1
:106ED2001D1D7FF37F7F497F7F617F11C70FFF8178
:106EE20057C04E4E7FF97F7F647F7F707F48E347B4
:106EF200FFC06BFFFF1DFFFF8D0D490D830D5F2549
:106F02005F25FF0511FF0507FF3307FF4907FF91C3
:106F120081230D25811D1D43430D11430D07430D93
:106F2200FF498DFFFF4EFFFFC6466446C1466F52C2
:106F32006F52FF4248FF4243FF5943FF6443FFC879
:106F4200C0514652C04E4E61614648614643614659
:106F5200FF64C68D118F0F25251DF38F11F3F311D9
:106F6200F34943F3F3815F0F43118D0711C74325A3
:106F72008D438D1319195F19F357258119138DFF4D
:106F82008D43071343078DEF1D1D115757134357A9
:106F92008D43571325578D251119191981251981EB
:106FA2005719114311C70F81C7F381C7492513F33D
:106FB200258F818F818D43F325830F0F430D1D1D77
:106FC200118D114343250D0F1D1125C648C7475288
:106FD200524EF9C748F9F948F96461F9F9C06F47A7
:106FE2006148C64348E36152C661C6494C4C6F4C86
:106FF200F96B52C04C49C6FFC66143496143C6F7AB
:107002004E4E486B6B49616BC6616B49526BC652FF
:10701200484C4C4CC0524CC06B4C486148E347C092
:10702200E3F9C0E3645249F952C7C0C7C0C661F967
:1070320052C1474761464E4E48C648616152464773
:047042004E48520062
:10B53B00C15AC152C139C13E017A00C138C14FC194
:10B54B00C741002700410028004200180000C14AF3
:10B55B00C159C1C9C1D1025C0000C154C13CC1BABF
:109BE200E4F52EF52F12C30B90014E7463F0E4904E
:109BF200014DF0900006F0F56C9001197412F0120C
:109C0200B4B99001327404F0129AA11259A4C25349
:109C120090008BE0FF7E007C007D3C12566D900030
:109C220000EEF0A3EFF0E49000E7F0A3F0C24ED212
:109C32004690001FF0A3F090004C74FAF0E49000FC
:109C4200CAF0A3F0C23DF551129E46129D1612C3F0
:109C52000B306923C269E50FD394004006D50F0388
:109C6200E4F50BE510D3940040021510E5126007ED
:109C7200E510700312C19DE551D39427406CE4F5C1
:109C820051D25A90014DE0D394004005E014F08087
:109C920002C267E4F559AF59EF3395E0FE74B32F72
:109CA200F58274003EF583E06035AD59ED3395E001
:109CB200FC74B32DF58274003CF583E014F074B3A8
:109CC2002DF58274003CF583E0701474992FF582AF
:109CD20074003EF583E0F52EF52FAF2F12748D053B
:109CE20059C3E5596480949740AC900028E0700312
:109CF200029C4A14F0E024B0F582E43400F583E0DB
:109D0200F554248DF582E43400F583E0F52FFF123B
:049D1200748D80D6F6
:10B4B900D294C2D812C24D12C30BD2A5D2A4C2A033
:10B4C900C2A1C2A2C2A3C29243BF02D2DBD2DA7521
:10B4D900985075892175CDFC75CC6675CBFC75CAFC
:10B4E90066C2CDC2CCC2CBC2C9C2C8C2CAD2AD75AE
:10B4F9008DFD758BFDE4F58A758C80D28ED28CD248
:10B50900A9D28AD2AAD2ACD2AFD2B9D2BC1294EF04
:10B519009000D6E0D3940350037525FF7F5612BEE1
:10B5290002EF6007758780750C0322E4F587750CB7
:02B539000622E8
:10C13E00205316900030E06010E4FD7F1212BF6EA7
:0AC14E00D253900030E0787AF62218
:1059A400755A00755B4E9000AE7427F09000AC748D
:1059B40025F0A304F09000AF7429F012C1B1E49073
:1059C40000D3F0FD7F7212BED67F0512BE02BF0166
:1059D4000A7F0412BE02EF6429602C900037740120
:1059E400F0E490003BF0D23E127BB87D017F0512BB
:1059F400BED67D297F0412BED6E490013AF0FD7F25
:105A0400FF12BED6025B5A7F5F12BE0290003BEFCC
:105A1400F0D394014002E4F0E4F530F531E53124AB
:105A24004FFF12BE02AD31742B2DF582E43400F524
:105A340083EFF0E53125E0FFE53033FE90003BE0F5
:105A440075F0C4906BFA125877E5822FF582E583DE
:105A54003EF583E493FC742B2DF582E43400F58346
:105A6400E0D39C403B90003BE075F0C4906BFA128D
:105A74005877E5822FF582E5833EF583E493FFAE04
:105A840031742B2EF582E43400F583EFF0EE244FCD
:105A9400FF742B2EF582E43400F583E0FD12BED6AC
:105AA400E53125E0FFE53033FE90003BE075F0C4BE
:105AB400906BF9125877E5822FF582E5833EF583E2
:105AC400E493FD742B2531F582E43400F583E0C3BF
:105AD4009D503B90003BE075F0C4906BF9125877F1
:105AE400E5822FF582E5833EF583E493FFAE3174BE
:105AF4002B2EF582E43400F583EFF0EE244FFF748F
:105B04002B2EF582E43400F583E0FD12BED6E53198
:105B1400244FFFE43530FEEF646A4E6006EF646B99
:105B24004E701D900027E07017E531244FFFE4FD0F
:105B340012BED6742B2531F582E43400F583E4F0EB
:105B44000531E53170020530C39462E53064809418
:105B5400805003025A21E4FF12BE0290001AEFF0B3
:105B64007F0112BE0290001BEFF07F0212BE029072
:105B7400001CEFF07F0312BE0290001DEFF09000B6
:105B84003AE0FF900039E02FFFE433CF240ACF340A
:105B940000FE900035E0C39FEE6480F87480985056
:105BA4001690003AE0FF900039E02F240A90003567
:105BB400F0FD7F5912BED67F4E12BE02EF7F00FE6B
:105BC400C006C0077F4D12BE02EFFDD0E02DFED00F
:105BD400E0340090011EF0A3CEF07F4812BE02EF25
:105BE4007F00FEC006C0077F4712BE02EFFDD0E073
:105BF4002DFED0E03400900120F0A3CEF07F4A12B5
:105C0400BE02EF7F00FEC006C0077F4912BE02EF4E
:105C1400FDD0E02DFED0E03400900122F0A3CEF0C0
:105C24007F4C12BE02EF7F00FEC006C0077F4B12FE
:105C3400BE02EFFDD0E02DFFD0E03400FE90012441
:105C4400F0A3EFF0D394E8EE94035009C390012439
:105C5400E0940050179001247401F0A374F4F0FD53
:105C64007F4B12BED67D017F4C12BED690011EE042
:105C7400FEA3E0D394E8EE94035006C3EE940050E0
:105C84001790011E7401F0A374F4F0FD7F4D12BE51
:105C9400D67D017F4E12BED6900122E0FEA3E0D352
:105CA40094E8EE94035006C3EE940050179001223A
:105CB4007401F0A374F4F0FD7F4912BED67D017F18
:105CC4004A12BED6900120E0FEA3E0D394E8EE94FD
:105CD400035006C3EE940050179001207401F0A302
:105CE40074F4F0FD7F4712BED67D017F4812BED604
:105CF4007FFF12BE0290013AEFF0900037E0F558B2
:105D0400E5587002C2AA900043E014600E24FE60BD
:105D1400172403701FE49000538012900053E07026
:105D240013900053740480059000537404F0FD7FB5
:105D34007712BED690008BE06009E4FD7F1512BF98
:105D44006EC23A900053E0900132F090002AF07F46
:105D54000912BE028F327F0A7E0012C251E5323030
:105D6400E4077F0912BE028F32E53220E438900046
:105D74007FE06402600CA3E064026006A3E06402B6
:105D84007024900030E0D39400401BE490002AF08B
:105D9400900053F0FD7F7712BED6C24D53570EAD1F
:105DA400577F0912BED690002AE0D394004005D252
:105DB4006612C13E1297E5900072E0B4011BD2CA8C
:105DC40090000212584600000000E4FD7F0412BF58
:105DD4006E78797602D2238007C2CA7F0412C27811
:105DE400900083E07006900082E0600C900085E0F3
:105DF400700A900084E07004C254801DD254C23CE6
:105E0400900085E0FE900084E07C002400FFEC3EDE
:105E1400FEE4FD9000071258217F6F12BE02BF02FC
:105E240002D2687B017A01793B7F067EEF12C2B60B
:105E340090013BE0FFF46003EF70207F0612BE0286
:105E440090013BEFF07F0612BE02EF60087F06125E
:105E5400BE02BFFF0690013B74FEF090013BE0FDE3
:105E64007F0612BED630480312BA6A12C30BE4F599
:105E740030F531F5327FD07E0712C25112B15BEF9B
:105E84002531F531EE3530F5300532E532C3940570
:105E940040E3AE30AF317C007D051256D48E308F96
:105EA40031D3E53194F2E530648094834004D259CF
:105EB4008002C25930590990002BE0701B048011F4
:105EC4009000D6E0C39403500F90002BE0B4020876
:105ED400E4F0FD7F4F12BED630480990014EE070C9
:105EE4000312BA6A90014EE0C394035004C23B808B
:105EF40002D23B124025E4F53274FB2532F582E4EC
:105F04003400F583E4F074D72532F582E43400F5E7
:105F140083E4F00532E532B403DF7F3012BE02EFD2
:105F24007F00FEC006C0077F2F12BE02EFFDD0E047
:105F34002DFFD0E03400FEC006C0077F1C12BE0255
:105F4400EF7F00FEC006C0077F1B12BE02EFFDD02C
:105F5400E02DFDD0E03400FCD007D006C3ED9FEE69
:105F64006480F8EC64809850089000E97401F08033
:105F740005E49000E9F07F4612BE02EF7F00FEC008
:105F840006C0077F4512BE02EFFDD0E02DFFD0E032
:105F94003400FEC006C0077F3212BE02EF7F00FE4F
:105FA400C006C0077F3112BE02EFFDD0E02DFDD048
:105FB400E03400FCD007D006C3ED9FEE6480F8EC1B
:105FC40064809850089000EA7401F08005E4900021
:105FD400EAF030572012C2ED12BD5A12C22E12C17D
:105FE400D71281C812BACA9001197412F0D26D1274
:105FF40032EC12028C12C26A90002AE070075357E6
:10600400FEC24D8005435701D24D535703AD577F10
:106014000912BED69000AB7424F012B874E47BFF6E
:0E6024007A7FF9F812BC99AE02AF0302BD14E8
:10C15800900028E0C394035010E0FE04F074B02E61
:0AC16800F582E43400F583EFF022C5
:10C1B100E4FF74B32FF582E43400F583E4F00FBF9C
:02C1C10017F075
:01C1C3002259
:0ABF64009000A0740FF0E4FD7F07C9
:10BF6E00ED7013EF906BE293FE74B32FF582E43411
:10BF7E0000F583EEF02274B32FF582E43400F583DE
:03BF8E00EDF022B1
:0DC2780074B32FF582E43400F583E4F02266
:10748D00C260EF125883750C00750F01766E02768F
:10749D006203766804767105765F06761D07760BB6
:1074AD0008760E0976110A76140B76170C761A0DDE
:1074BD0076200E76420F764410764711764A127674
:1074CD004D13765014765315765916766B177674D0
:1074DD001A76771B767D1C769A1D76B71E76D41F8D
:1074ED0076F120770D21772722775023777A24772D
:1074FD00C72577E32677E6277835290000785202ED
:10750D0081C8303D16900021E004F0E0D394354061
:10751D000AE4F0055DE55D7002055C20540302751B
:10752D00E3900086E0FB70028030EBB40110900018
:10753D0029E004F0E0D39435403CE4F0801C900049
:10754D0029E004F0E0D39435402CE4F09000CCE039
:10755D0004F0E0D3943B401EE4F09000071258096C
:10756D00EF24FFFFEE34FFFEED34FFFDEC34FFFCA6
:10757D00900007125821E4FFFEFDFC900007125801
:10758D0015C31257F87020203C1D900083E0FE902B
:10759D000082E07C002400FFEC3EFEE4FD9000073D
:1075AD00125821D23C802FE4FFFEFDFC9000071203
:1075BD005815C31257F8701E303C1B900085E0FE25
:1075CD00900084E07C002400FFEC3EFEE4FD900082
:1075DD0007125821C23C305D22D3900111E0940076
:1075ED00900110E09400401374FFF5F012570A90CB
:1075FD000110E07002A3E07002C25D029F7502A847
:10760D001A02994502A08C02AE9802B0BE02AAA839
:10761D0002916A90004AE07005C24A02BEA3900032
:10762D004AE0FF64026008EF6403600302785212BF
:10763D00BEA3D24A22801802B63602B6B202AC40C0
:10764D00028D7B02845712704C02AB7612704C0285
:10765D00C21E02C1FC1232ECD24E2202C1C402BDC6
:10766D005A02028C02499502892675120302C19DA8
:10767D009000E2E014F0E0700D7B017A0079E7C232
:10768D00647D01027770E4FD7F0A02784F9000E37C
:10769D00E014F0E0700D7B017A0079E7C2647D03A0
:1076AD00027770E4FD7F0B02784F9000E4E014F058
:1076BD00E0700D7B017A0079E7C2647D0502777079
:1076CD00E4FD7F0C02784F9000E5E014F0E0700DC2
:1076DD007B017A0079E7C2647D07027770E4FD7F54
:1076ED000D02784F9000E6E014F0E0700C7B017A0B
:1076FD000079E7C2647D09806AE4FD7F0E02784F50
:10770D00E4F5307B017A007918C264AD3012B80708
:10771D000530E530C3940240EA2290001EE004F0EB
:10772D00E0C394064016E4F090010CE014F0E07014
:10773D000B7B017A017902C264FD8027E4FD7F1085
:10774D0002784F900017E004F0E0C394064017E470
:10775D00F090010AE014F0E0700C7B017A017900E1
:10776D00C264FD02B807E4FD7F1102784F90000658
:10777D00E004F0E0C39406403AE4F0787AE6D3945E
:10778D0000400116787AE6702AC253304D033066F8
:10779D0019C266C24DE490002AF0900053E09001AA
:1077AD0032F0E4900053F0FD8061435710AD577FE8
:1077BD0009805AE4FD7F1202784F7F0812BE02EF56
:1077CD0060030278527F0812BE02EF7078439B105F
:1077DD0075A5C3F5A322D25E2290000074FFF5F0CB
:1077ED0012570A900000E07002A3E07023203A20A7
:1077FD00D24D43570190002A7404F0AD577F091202
:10780D00BED690002AE0FD900053F07F7702BED6E1
:10781D00D3900001E09400900000E09400402620F9
:10782D003A23E4FD7F15801A9000D3E0FF04F0EFBA
:10783D00D39409E44009F07F1612C278D26822FD74
:05784D007F1612BF6E62
:017852002213
:10BACA0090004AE0B4031290008E7464F0A3F0A3CD
:10BADA00F0A3F0A3F0A3F08031900044E090008E30
:10BAEA00B406107464F0A3F0A3F0A3F0900093746A
:10BAFA000980117408F0A304F0A304F0A304F090E1
:10BB0A000093740DF090009214F0900096740EF069
:0CBB1A0012C22E12C1D7E4900119F022D3
:10C0380090008EBF030E7464F0A3F0A3F0A3F0A3E6
:10C04800F0A3F0227408F0A304F0A304F0A304F012
:07C05800A304F0A304F02291
:109AA100E4F530900022E0FE75F030A424FEF5824A
:109AB100E4346EF583E493FFEE75F030A424FFF5F2
:109AC10082E4346EF583E493FD900022E075F0307A
:109AD100A42400F582E4346FF583E493FB12C28B76
:109AE10012C24D12C30B12C24D12C30B12C24D1240
:109AF100C30B12C24D12C30B900022E0FE75F0148D
:109B0100A424ABF582E4346EF583E493FFEE75F0A3
:109B110014A424BCF582E4346EF583E493FD900033
:109B210022E075F014A424B0F582E4346EF583E4E8
:109B310093FB12C28B12C30B12C24D12C30B12C282
:109B41004D12C30B12C24D12C30B7F0912BE028FFD
:109B510057E5BF30E70543570280035357FDAD5723
:109B61007F0912BED6C2577F0A12BE028F307E0015
:109B710012BD1412BCDD7C017D2C1256D4EF04F50C
:109B810030FD7F0A12BED67F0A12BE02EF65306039
:109B910047900022E0FE75F030A424FBF582E43406
:109BA1006EF583E493FFEE75F030A424FCF582E4B6
:109BB100346EF583E493FD900022E075F030A42427
:109BC100FDF582E4346EF583E493FB12C28B12C27D
:109BD1004D12C30BC2508002D2577F327E0002C2A7
:019BE1005132
:10A28600900140EEF0A3EFF0C39464EE94005046C4
:10A296007520FF900140E0FAA3E0FB7C007D0AFFF9
:10A2A600AE0212567F900022E075F014A424B3F596
:10A2B60082E4346EF583E5822FF582E5833EF583ED
:10A2C600E493F5217C007D0AAF03AE0212567F901F
:10A2D6000022E002A362900140E0FAA3E0FB7C03C7
:10A2E6007DE8FFAE0212567F7E007F64CFCDCFCED3
:10A2F600CCCE12567F900022E075F014A424A9F566
:10A3060082E4346EF583E5822FF582E5833EF5839C
:10A31600E493F5207C007D64AF03AE0212567F7E87
:10A32600007F0ACFCDCFCECCCE12567F900022E052
:10A33600FB75F014A424B3F582E4346EF583E5824C
:10A346002FF582E5833EF583E493F521900140E005
:10A35600FEA3E0FF7C007D0A12567FEB75F014A485
:10A3660024A9F582E4346EF583E5822DF582E58332
:0AA376003CF583E493F522028926EA
:09AF5300E47B0AFAF9F812BC993A
:10AF5C00AB07AA067520FF7521FF7C037DE812560E
:10AF6C007F7E007F64CFCDCFCECCCE12567FEF4EFE
:10AF7C00601F900022E075F014A424A9F582E4343B
:10AF8C006EF583E5822FF582E5833EF583E493F538
:10AF9C00207C007D64AF03AE0212567F7E007F0AD8
:10AFAC00CFCDCFCECCCE12567FEF4E7005E520F430
:10AFBC00601F900022E075F014A424A9F582E434FB
:10AFCC006EF583E5822FF582E5833EF583E493F5F8
:10AFDC0021AE02AF037C007D0A12567F900022E066
:10AFEC0075F014A424A9F582E4346EF583E5822D62
:0EAFFC00F582E5833CF583E493F52202892675
:06C285007BFF7DFF7FFF3F
:07C28B008F208D218B222280
:10A47400C3E49FFFE49EFE900140F0A3EFF0C39479
:10A4840064EE9400407475207F900140E0FAA3E0EC
:10A49400FB7C037DE8FFAE0212567F7E007F64CF13
:10A4A400CDCFCECCCE12567F900022E075F014A40E
:10A4B40024A9F582E4346EF583E5822FF582E583E1
:10A4C4003EF583E493F5217C007D64AF03AE021274
:10A4D400567F7E007F0ACFCDCFCECCCE12567F9052
:10A4E4000022E075F014A424B3F582E4346EF583FD
:10A4F400E5822FF582E5833E805875207F900140E8
:10A50400E0FAA3E0FB7C007D0AFFAE0212567F90C6
:10A514000022E075F014A424B3F582E4346EF583CC
:10A52400E5822FF582E5833EF583E493F5217C00F3
:10A534007D0AAF03AE0212567F900022E075F0143C
:10A54400A424A9F582E4346EF583E5822DF582E531
:0BA55400833CF583E493F52202892686
:10A81A0020520302A8F6E55B64F5455A60061291D8
:10A82A006A02A8F6900045E06402603690004BE0A8
:10A83A00FFC394034006EFD39404400E90007BE0DC
:10A84A00787626F618E436F6801890004BE0FFC3B7
:10A85A009403400EEFD394045008787606E61870F5
:10A86A00010690004BE0FFC394034006EFD3940423
:10A87A004025900048E0FF7E007C007D0A12566D5C
:10A88A00D37876E69FEE6480F5F018E6648095F05A
:10A89A004005A60608A6077875E6F53108E6F532FA
:10A8AA00D394E7E53164809483400DAE31AF327CB6
:10A8BA00007D0A1256D4802290004BE0FFC3940315
:10A8CA00401DEFD394045017C3E53164809480AFE0
:10A8DA0032AE31500512A474800C12AF5C8007AFFF
:0FA8EA0032AE3112A28612BF6A02C23E12A380A2
:01A8F900223C
:10994500205203029A9DE55B64F5455A6006129123
:109955006A029A9D900045E06402603A90004BE0EF
:10996500FFC394034006EFD39404401290007BE0BC
:10997500FFC37876E69FF618E69400F68018900007
:109985004BE0FFC39403400EEFD394045008787660
:10999500E6161870011690004BE0FFC394034009CA
:1099A500EFD394045003029A48900051E0FB240140
:1099B500FFE433FE7C007D0A12566DC37876E69F80
:1099C500EE6480F5F018E6648095F0401F9000493C
:1099D500E02401FFE433FE12566DC37876E69FEE70
:1099E5006480F5F018E6648095F05057900044E0E7
:1099F5006403702A900049E02401FFE433FEEBC3C1
:109A05009FEE6480F874809850028007900051E0C2
:109A1500FF7E007C007D0A12566D787580209000CF
:109A250049E0FF7E007C007D0A12566DC37876E61C
:109A35009FEE6480F5F018E6648095F05005A60663
:109A450008A6077875E6F53108E6F532D394E7E51B
:109A55003164809483400DAE31AF327C007D0A12B3
:109A650056D4802290004BE0FFC39403401DEFD3F2
:109A750094045017C3E53164809480AF32AE315001
:109A85000512A474800C12AF5C8007AF32AE3112A0
:0B9A9500A28612BF6A02C23E12A3802C
:019AA00022A3
:10A08C00900044E0B4020CC24412028CE4FD7F0840
:10A09C0002BF6E900044E06403600302A189205269
:10A0AC000302A180E55B64F6455A600612916A02D0
:10A0BC00A180900045E06402600C90007BE0787613
:10A0CC0026F618E436F690004FE0FBFF7E007C008D
:10A0DC007D0A12566DD37876E69FEE6480F5F01803
:10A0EC00E6648095F05020900048E024FFFFE434B3
:10A0FC00FFFE12566DD37876E69FEE6480F5F0186D
:10A10C00E6648095F0402B900048E0FF14FEEBD302
:10A11C009E400AEF24FFFFE434FFFE800790004FBF
:10A12C00E0FF7E007C007D0A12566D7875A606084D
:10A13C00A6077875E6FE08E6FFEE3395E08F348EC1
:10A14C0033F532F531E47FE77E03FDFCAB34AA3303
:10A15C00A932A831D31257E2400DAF34AE33AD3231
:10A16C00AC3112AF538007AE33AF3412A28612BF9C
:0DA17C006A02C23E755A00755BF612A3869A
:01A1890022B3
:10AE9800900044E0B4020CD24412028CE4FD7F0816
:10AEA80002BF6E900044E06403600302AF52205278
:10AEB8000302AF49E55B64F6455A600612916A02DF
:10AEC800AF49900045E06402601090007BE0FFC34A
:10AED8007876E69FF618E69400F6900049E0FF7E43
:10AEE800007C007D0A12566DC37876E69FEE64807A
:10AEF800F5F018E6648095F05005A60608A60778D0
:10AF080075E6FE08E6FFEE3395E08F348E33F532B2
:10AF1800F531E47FE77E03FDFCAB34AA33A932A800
:10AF280031D31257E2400DAF34AE33AD32AC3112EB
:10AF3800AF538007AE33AF3412A28612BF6A02C283
:0AAF48003E755A00755BF612A386F1
:01AF520022DC
:10B0BE00900044E0700302B15AC26C20520302B1F8
:10B0CE0051E55B64F7455A600512916A8075787692
:10B0DE0006E618700106D37876E6940418E66480C6
:10B0EE009480400D900044E0B40406E4F608F68027
:10B0FE0033900045E0FFB4010478758022EFB4026E
:10B10E000A7876E61618701C16801990003CE0FF3F
:10B11E00D37876E69F7480F5F0186695F040057644
:10B12E00000876047876E6FF12B00A7876E690008C
:10B13E002AF012028CE4FD7F0812BF6E1F12BF6E42
:0DB14E0002C23E755A00755BF712A38622FF
:10AAA800900044E0B40413304404C2448002D24409
:10AAB80012028CE4FD7F0802BF6E900044E0FF7034
:10AAC8000302AB756405700302AB75C26C205203B8
:10AAD80002AB6CE55B64F7455A600612916A02ABFB
:10AAE8006C7876E61618700116900045E0FFB40100
:10AAF80008E47875F608F6804CEFB4020A78760612
:10AB0800E618704106803E90003BE075F0C4906CFA
:10AB180049125877E493FF7E00C37876E69F7480E5
:10AB2800F5F0186695F05002801690003CE0FF7E24
:10AB380000D37876E69F7480F5F0186695F04005A6
:10AB4800A60608A6077876E6FF12B00A7876E69099
:10AB5800002AF012028CE4FD7F0812BF6E1F12BF9C
:0EAB68006E02C23E755A00755BF712A386227C
:10B00A00AE07EE6404701090003CE0601B900045AF
:10B01A00E0604E8013804A7876E6640118467041F3
:10B02A0090003CE064017039900022E0FD75F01256
:10B03A00A424E0F582E4346EF583E493FFED75F021
:10B04A0012A424E1F582E4346EF583E493FD9000C2
:10B05A0022E075F012A424E2F582E4346EF58380CE
:10B06A004C900022E0FD75F012A424D1F582E4345C
:10B07A006EF58375F003EE125877E493FFED75F0E1
:10B08A0012A424D2F582E4346EF58375F003EE122D
:10B09A005877E493FD900022E075F012A424D3F5CA
:10B0AA0082E4346EF58375F003EE125877E493FB6D
:04B0BA0012C28B2211
:06A38000755A00755BF543
:10A38600D2527F0112C278E55A600302A464E55BEB
:10A39600240A607C14700302A4532402600302A4FE
:10A3A6006490004BE0FFC394034006EFD39404404F
:10A3B6000A900050E0FE90004F800890005EE0FE9C
:10A3C60090005DE07C002400F536EC3EF5357875AE
:10A3D600A63508A636D3E53694E7E535648094833A
:10A3E6004008AE35AF367C00805090004BE0FFC38E
:10A3F60094034050EFD39404504AC3E535648094E7
:10A4060080AF36AE35503812A47480528031803415
:10A41600900052E0FE900051E07C002400F536ECFE
:10A426003EF5357875F608A636D3E53694E7E53574
:10A4360064809483400EAE35AF367D0A1256D41230
:10A44600AF5C801AAF36AE3512A2868011900053EB
:10A45600E0FF7875760008A607E6FF12B00A12C27A
:0EA466003E9000A07407F0E4FD7F0702BF6E79
:10916A00E55A6003029307E55B240A700302922D15
:10917A001470030292C02402600302930790004B0A
:10918A00E0FFC394034006EFD3940440727876E676
:10919A0090004FF018E6FF3395E0EFA3F090004FF0
:1091AA00E0FD7F7312BED6900050E0FD7F7412BEC0
:1091BA00D6900044E064016003029307900050E0F7
:1091CA00FE90004FE07C002400FFEC3EFE90003A47
:1091DA00E0FDC3EF9DFFEE9C90013EF0A3EFF090FF
:1091EA00013EE0900052F090013FE0900051F0FD06
:1091FA007F7512BED6900052E0FD7F760292BB7850
:10920A0076E690005DF018E6FF3395E0EFA3F09064
:10921A00005DE0FD7F8112BED690005EE0FD7F8298
:10922A000292BB7876E6900051F018E6FF3395E09B
:10923A00EFA3F0900051E0FD7F7512BED690005268
:10924A00E0FD7F7612BED6900052E0FE900051E01B
:10925A00F97C002400FDEC3EFC900050E0FE9000FA
:10926A004FE07A002400FFEA3EFED3EF9DEC6480D3
:10927A00F8EE6480984003029307900052E0FEE9FA
:10928A007C002400FFEC3ECF240ACF340090013E3C
:10929A00F0A3EFF090013EE0900050F090013FE023
:1092AA0090004FF0FD7F7312BED6900050E0FD7F14
:1092BA007412BED68047900053E0900132F078765F
:1092CA00E6900053F0E690002AF0E6FD7F7712BEA2
:1092DA00D690002AE070145357FEC24DAD577F094D
:1092EA0012BED6C253E4787AF6800F20530C435745
:1092FA0001D24DAD577F0912BED61297E57F0712EC
:10930A00C278C25212C2C290004AE0B4032412BF09
:10931A0064E55B64F5455A7007F55A755B74800D10
:10932A00E55B64F7455A7005F55A755B7512AB76BD
:07933A00800312BACAD26DD4
:019341002209
:10C1FC00B2393039047D0380027D057F0612BF6E93
:01C20C00220F
:0FC23E0090009F7406F07D03FF12BF6E056C2207
:0BC2C2007F0612C278C239E4F56C223E
:10BEA30012C2C29000A0740FF0304A17755A007581
:10BEB3005B4E90004AE0B40306755A00755B74C28A
:10BEC300428008755A00755B4ED24212AB767F01F1
:03BED30002C27830
:10C21E007F0712C27812C2C212BACAC252C26522B5
:10B63600E55B6472455A700C204A09F55A755B4EF3
:10B64600D2428065304A4B90004AE064037039E587
:10B656005B6474455A7007F55A755B758030E55B17
:10B666006475455A7007F55A755B4E8021E55B6433
:10B676004E455A7004F55A8012E55B6454455A707B
:10B686000DF55A755B748006755A00755B54C24297
:10B696008017E55B644E455A7007304204C242800B
:0CB6A60008055BE55B7002055A02AB76FC
:10B6B20012AB76304A4990004AE064037039E55B88
:10B6C2006474455A7007F55A755B548058E55B649B
:10B6D20054455A7004F55A8021E55B644E455A7010
:10B6E20007F55A755B75803DE55B6475455A7035A3
:10B6F200F55A755B74802E755A00755B4E8026E58F
:10B702005B644E455A700A304207F55A755B728087
:10B7120014E55B644E455A7004D2428008E55B151D
:08B722005B7002155A02AB76C0
:10785300E55A6003027BADE55B12588378C34E792A
:10786300894F7989507989517989527989537989ED
:10787300547B65557B935679895779895879895B08
:1078830079895C79155F7989607989617989627908
:10789300896379896479896579896679896779934F
:1078A3006879896979896A79896B79896C79896D4C
:1078B3007B6B6E79896F7AE2717AE27200007BAD3D
:1078C3003042030279897875E6F53108E6F532D35B
:1078D30094E7E531648094834031AE31AF327C006C
:1078E3007D0A1256D4AB05AE31AF327C007D0A124D
:1078F30056D48E318F32EBC3940540080532E532FE
:1079030070020531AF32AE31027B90AF32AE31023D
:107913007BB47876E618469000226035E0FE75F079
:1079230030A424F5F582E4346EF583E493FFEE7519
:10793300F030A424F6F582E4346EF583E493FD90ED
:107943000022E075F030A424F7F582E4346E027B64
:107953005DE0FE75F030A424F8F582E4346EF5831F
:10796300E493FFEE75F030A424F9F582E4346EF568
:1079730083E493FD900022E075F030A424FAF582AD
:10798300E4346E027B5D7875E6FE08E6FF027B90C9
:107993007875E6FE08E6FFEE6003027BB7EF125848
:1079A3008379BD0079C40179CB027A03037A3B045E
:1079B3007A73057AAB0600007BB77F027E00027BF9
:1079C300907F047E00027B90900022E0FE75F030F1
:1079D300A42404F582E4346FF583E493FFEE75F099
:1079E30030A42405F582E4346FF583E493FD90001D
:1079F30022E075F030A42406F582E4346F027B5D47
:107A0300900022E0FE75F030A42407F582E4346F81
:107A1300F583E493FFEE75F030A42408F582E43493
:107A23006FF583E493FD900022E075F030A4240900
:107A3300F582E4346F027B5D900022E0FE75F03046
:107A4300A4240AF582E4346FF583E493FFEE75F022
:107A530030A4240BF582E4346FF583E493FD9000A6
:107A630022E075F030A4240CF582E4346F027B5DD0
:107A7300900022E0FE75F030A4240DF582E4346F0B
:107A8300F583E493FFEE75F030A4240EF582E4341D
:107A93006FF583E493FD900022E075F030A4240F8A
:107AA300F582E4346F027B5D900022E0FE75F030D6
:107AB300A42422F582E4346FF583E493FFEE75F09A
:107AC30030A42423F582E4346FF583E493FD90001E
:107AD30022E075F030A42424F582E4346F807B78AF
:107AE30075E6FE08E6FF7C007D021256D4ED4C904D
:107AF30000226034E0FE75F030A42410F582E434F3
:107B03006FF583E493FFEE75F030A42411F582E45E
:107B1300346FF583E493FD900022E075F030A424E4
:107B230012F582E4346F8032E0FE75F030A4241342
:107B3300F582E4346FF583E493FFEE75F030A4240B
:107B430014F582E4346FF583E493FD900022E0752D
:107B5300F030A42415F582E4346FF583E493FB023B
:107B6300C28B7F647E0080497876E618467004FFF6
:107B7300FE801A7876E66401184670057F01FE8060
:107B83000C7876E664021846702A7F02FE02AF5C28
:107B93007876E6184670057F60FE80157876E66491
:107BA300011846700F7FC0FE80077875E6FE08E671
:047BB300FF12A28695
:017BB70022AB
:10AB76009000917412F0900090F090008EF0A3F087
:10AB860090009314F090009214F0E55B644E455AE1
:10AB9600703A304237900022E0FE75F078A424C463
:10ABA600F582E4346FF583E493FFEE75F078A42420
:10ABB600C5F582E4346FF583E493FD900022E075D9
:10ABC600F078A424C6F582E4346F805F900022E01A
:10ABD600FE75F078906E6B12587775F003E55B1290
:10ABE6005877E55A75F003A42583F583E493FF753A
:10ABF600F078EE906E6C12587775F003E55B12589C
:10AC060077E55A75F003A42583F583E493FD900058
:10AC160022E075F078906E6D12587775F003E55B5B
:10AC2600125877E55A75F003A42583F583E493FB60
:0AAC360012C28BE4FD7F0702BF6E1F
:10AC4000E55B6474455A701290008E7408F0A3049A
:10AC5000F0A304F0A304F0A3801DE55B6475455ADE
:10AC6000701B900090740CF0A304F090008FF09093
:10AC7000008E14F09000927407F0A3F0229000A0D0
:10AC80007416F090009214F0A3F09000907413F0FA
:10AC9000A304F090008FF090008E1412BF69E55B62
:10ACA000644E455A701130420E90013BE0FF7875BA
:10ACB000760008A607801274DC255BF582E434FF79
:10ACC000F583E07875760008F6E55B644E455A70CA
:10ACD0002A2042279000D4E555F0A3E556F0787578
:10ACE000A65508A656C3E55564809480500DC3E46C
:10ACF0009556FFE4955518F608A607E55B6455459B
:09AD00005A7002D2561278532257
:108D7B0012BF6AE55B6466455A600BE55B646D4543
:108D8B005A6003028E26E55B6466455A704290007A
:108D9B0048E0FFC37876E69F7480F5F0186695F08F
:108DAB004003028F6490003BE075F0C4906C281276
:108DBB005877E493FFC308E69F7480F5F018669527
:108DCB00F04003028F640806E618704C06028F61B0
:108DDB00900048E024FFFFE434FFFEC37876E69F63
:108DEB00EE6480F5F018E6648095F04003028F6422
:108DFB0090003BE075F0C4906C36125877E493FF0B
:108E0B00C308E69F7480F5F0186695F04003028F57
:108E1B00640806E618700106028F61E55B646A451B
:108E2B005A6008E55B646B455A7009900027E07047
:108E3B0003028F61E55B644E455A7024304221C3B7
:108E4B007876E694FE18E66480948050090806E66E
:108E5B0018700A06800778757600087601028F6114
:108E6B00E55B645C455A705B7876E6184670189043
:108E7B000044E0FF64036006EFD39401500978755A
:108E8B0076000876028039E55B25E0FFE55A33FE74
:108E9B0090003BE075F0C4906B5C125877E5822F25
:108EAB00F582E5833EF583E493FFC37876E69F7402
:108EBB0080F5F0186695F050070806E61870010665
:108ECB00028F61E55B644E455A700D20420A78763D
:108EDB0006E618700106807EE55B6453455A7022E6
:108EEB0090003BE075F0C4906CA6125877E4937831
:108EFB007666700218E66008787606E6187001064A
:108F0B008054E55B25E0FFE55A33FE90003BE075AE
:108F1B00F0C4906B5C125877E5822FF582E5833EA7
:108F2B00F583E493787666700218E6602C78760603
:108F3B00E618700106E55B644F455A70197876E6C2
:108F4B0064021846701090014EE0C394035007085A
:108F5B00E61618700116127853E55B6455455A7086
:0D8F6B00087876E6900031F02212C23E2216
:1084570012BF6AE55B6466455A600BE55B646C4571
:108467005A6003028501E55B6466455A70429000D5
:1084770049E0FFD37876E69F7480F5F0186695F0AB
:1084870050030286C390003BE075F0C4906C27123E
:108497005877E493FFD308E69F7480F5F018669544
:1084A700F050030286C308E61618704B160286C002
:1084B700900049E02401FFE433FED37876E69FEE8F
:1084C7006480F5F018E6648095F050030286C39047
:1084D700003BE075F0C4906C33125877E493FFD3F8
:1084E70008E69F7480F5F0186695F050030286C37E
:1084F70008E616187001160286C0E55B6462455AE5
:108507006008E55B6461455A706EE55B6462455AD5
:1085170070337875E6FE08E6FF7C007D0A12566D1B
:10852700900039E0240AFDEC33FCD3EF9DEC648026
:10853700F8EE64809850030286C37876E6161870C2
:1085470001160286C07875E6FE08E6FF7C007D0A04
:1085570012566D90003AE0240AFDEC33FCD3EF9DF0
:10856700EC6480F8EE64809850030286C37876E660
:1085770016187001160286C0E55B645C455A706385
:10858700C37876E6940318E664809480400908E689
:108597001618704C1680497876E6640218467020E3
:1085A700900044E0FF64036006EFD394015008E4B1
:1085B7007875F608F68029787576000876018020A8
:1085C7007876E6640118467017900044E0FF64036C
:1085D7006006EFD3940150087876E61618700116F6
:1085E7000286C0E55B644E455A7024304221D37839
:1085F70076E6940118E664809480400908E6161828
:10860700700A168007787576000876FE0286C0E540
:108617005B644B455A7003304208E55B644D455A2D
:10862700700B7876E616187001160286C0E55B6453
:1086370053455A702290003BE075F0C4906CA51228
:108647005877E493787666700218E660087876E6DD
:1086570016187001168062E55B25E0FFE55A33FEC8
:1086670090003BE075F0C4906B5B125877E5822F62
:10867700F582E5833EF583E493787666700218E623
:10868700603A7876E61618700116E55B6451455A2C
:10869700700E90002BE0B40107787576000876011C
:1086A700E55B644F455A70117876E61846700A30D4
:1086B70059070806E618700106127853E55B6455FA
:1086C700455A70087876E6900031F02212C23E22B1
:10704C0012BF6412C2C2C256E55B6472455A701F0D
:10705C007875E6FE08E6FF7C007D021256D4ED4CF6
:10706C006003027488D23E127BB812C28580FEE5A2
:10707C005B6471455A70687875E6FE08E6FF7C0023
:10708C007D021256D4ED4C6003027488C2AFC2A9C3
:10709C00C2AAF59F7F7612C12212C30B7D007CEC35
:1070AC007F5512C0C87D017CEC7FAA12C0C8E47861
:1070BC008FF6788FE6FFC394F3501812BE027890C7
:1070CC00EFF618E62402FDE434ECFC12C0C8788F0D
:1070DC000680DF12C30BD2A9D2AAD2AF027488E504
:1070EC005B6455455A700A900031E0FD7F5502747F
:1070FC0085E55B644E455A60030272093042030217
:10710C00720990002BE07048C3E555648094809020
:10711C000011E0FEA3E0FF5012C3E49FFFE49EFECB
:10712C00C3EF787696FFEE18968009C37876E69FC3
:10713C00FF18E69E9001248FF012570A900125E06B
:10714C00FD7F4B12BED6900124E0FD7F4C027200F5
:10715C0090002BE06401704F90002DE064046047B8
:10716C00C3E5556480948090000BE0FEA3E0FF50D3
:10717C0012C3E49FFFE49EFEC3EF787696FFEE18F1
:10718C00968009C37876E69FFF18E69E90011E8FC5
:10719C00F012570A90011FE0FD7F4D12BED69001F0
:1071AC001EE0FD7F4E804D90002BE064027048C3C2
:1071BC00E5556480948090000FE0FEA3E0FF501230
:1071CC00C3E49FFFE49EFEC3EF787696FFEE18961D
:1071DC008009C37876E69FFF18E69E9001228FF017
:1071EC0012570A900123E0FD7F4912BED69001226E
:1071FC00E0FD7F4A12BED61281C8027488E55B643A
:10720C004E455A701F30421C7876E6FD7F0612BE42
:10721C00D67876E690013BF07D067CEFE4FF12C059
:10722C00C8027488E55B6453455A60030272C978DE
:10723C0076E6640518467013900038E0FF6402602F
:10724C0041EF6403603C7402F08031900038E0FF41
:10725C0064026005EF64037029900044E0FF64024F
:10726C006009EF64046004EFB40508900038740101
:10727C00F08005E4900038F0900038E0FD7F5C125F
:10728C00BED67876E664031846600808E6640418EF
:10729C0046700C9000437402F0FD7F6712BED690CE
:1072AC000081E0787666700218E6700302748878C4
:1072BC0076E6900081F0E0FD7FA502748574DC25F4
:1072CC005BF582E434FFF583E0787666700218E6AD
:1072DC0070030274887876E6FEAF5B74DC2FF5825F
:1072EC00E434FFF583EEF0E6FD12BED6E55B645B9D
:1072FC00455A700AD23E127BB812C28580FEE55BFD
:10730C00645F455A702E7F5612BE02788FA6077F97
:10731C004F12BE027890A607D23E127BB8788FE649
:10732C00FD7F5612BED67890E6FD7F4F12BED61268
:10733C00C28580FEE55B6468455A700512C2858083
:10734C00FEE55B6469455A702990002AF05357FE9C
:10735C00C24DAD577F0912BED6C253E4787AF6906F
:10736C000053E0900132F0E4900053F0FD7F77126F
:10737C00BED6E55B644F455A70199001197405F03F
:10738C0090002BE0B4010C90002D7401F0FD7F51A6
:10739C0012BED6E55B645C455A70597876E6640398
:1073AC001846600808E664021846701490002FE036
:1073BC006405600C9000817405F0FD7FA512BED6AB
:1073CC007876E664041846701190002DE064016034
:1073DC00097401F0FD7F5112BED67876E66405186B
:1073EC0046701190002EE0640160097401F0FD7F7D
:1073FC005212BED6E55B6456455A700512C28580A2
:10740C00FEE55B645D455A6008E55B645E455A7059
:10741C006BE55B645D455A703190003EE075F00A97
:10742C00A4FFC37876E69FE5F06480F5F018E66477
:10743C008095F04047E6FE08E6FF7C007D0A125678
:10744C00D4EF04F0E0FD7F62802F90003DE075F0FA
:10745C000AA4FFC37876E69FE5F06480F5F018E6A1
:10746C00648095F04016E6FE08E6FF7C007D0A126B
:10747C0056D4EF04F0E0FD7F6112BED6D26DC26C23
:01748C0022DD
:10BD9300E4F540E54030470C24B1FFE540906E45A3
:10BDA30093FD801724B3FFE434ECFE7B007A007923
:10BDB3004112C2B6E54024B1FFAD4112BED60540E3
:07BDC300E540C3942A40CCC7
:01BDCA002256
:10B79A003047197D017F0F12BED6E4FD7F1012BE1D
:10B7AA00D67D017F1112BED6E4FD804B7B007A0064
:10B7BA0079407F117EEC12C2B6AD407F0F12BED621
:10B7CA007B007A0079407F127EEC12C2B6AD407FD0
:10B7DA001012BED67B007A0079407F137EEC12C22B
:10B7EA00B6AD407F1112BED67B007A0079407F1435
:0CB7FA007EEC12C2B6AD407F1212BED62B
:01B80600221F
:10A9D60020470302AA7FE4F540E540C31325E0249F
:10A9E6006FF582E4346EF583740193FDE540241B14
:10A9F600FF12BED605400540E540C3941540DA7502
:10AA06004001E540C31325E0246FF582E4346EF57A
:10AA160083E493FDE540241BFF12BED605400540A6
:10AA2600E540C3941640DBE4F540E540C31325E05A
:10AA36002485F582E4346EF583740193FDE54024A4
:10AA460031FF12BED605400540E540C3941540DAF5
:10AA5600754001E540C31325E02485F582E4346E94
:10AA6600F583E493FDE5402431FF12BED60540058B
:10AA760040E540C3941640DB22E4F540E540241D42
:10AA8600FFE434ECFE7B007A00794112C2B6E54061
:10AA9600241BFFAD4112BED60540E540C3942C40B1
:01AAA600DBD4
:01AAA700228C
:10B72A00304744E4F540E4F541E54075F007A424C8
:10B73A009BF582E4346EF583E5822541F582E43592
:10B74A0083F583E493FDE54075F005A424E92541DA
:10B75A00FF12BED60541E541C3940740CC0540E53A
:10B76A0040C3940240C022E4F540E54024EBFFE4E4
:10B77A0034ECFE7B007A00794212C2B6E54024E935
:0FB78A00FFAD4212BED60540E540C3940A40DB36
:01B79900228D
:107BB8007B007A00793E7F007EEC12C2B67B007AA9
:107BC80000793F7F017EEC12C2B6E53EB45509E567
:107BD8003FB4AA04C2478002D2477F0512BE02BF43
:107BE800010A7F0412BE02EF64296004C2618002A8
:107BF800D26130381BE4F53D90003BF0FD7F5F1209
:107C0800BED69000377401F0FD7F5B12BED68006A9
:107C180090003BE0F53DE53DD394014003E4F53D9C
:107C2800203E09203806306103027CF7753C4F304E
:107C3800611BE53C645B7003027CEBE53C6472709D
:107C480003027CEBE53C645F7003027CEBE53C647B
:107C58006A6005E53CB46B1B900027E07015FDAF2A
:107C68003C12BED674DC253CF582E434FFF583E48F
:107C7800F0807030474675F062E53D906D321258DD
:107C880077E582253CF582E43583F583E493FDAFFF
:107C98003C12BED675F062E53D906D32125877E51C
:107CA80082253CF582E43583F583E493FF74DC2573
:107CB8003CF582E434FFF583EFF08027E53C2402AD
:107CC800FFE434ECFE7B007A00793E12C2B6AD3E8A
:107CD800AF3C12BED674DC253CF582E434FFF58354
:107CE800E53EF0053CE53CC394B15003027C3720E7
:107CF8003E03027D7BE4F53CE53C2415FFE434ECCF
:107D0800FE7B007A00793E12C2B6E53C2413FFAD33
:107D18003E12BED6053CE53CC3940840DB12C30BBB
:107D28007D707F1312BED67D307F1412BED67D6D56
:107D38007F1512BED67D707F1612BED67D707F1756
:107D480012BED67D307F1812BED67D6D7F1912BE49
:107D5800D67D707F1A12BED612BD9312C30B12BC09
:107D68000C12C30B12B72A12C30B12A9D612C30BDB
:107D780012B79A306106203803027EB53047753055
:107D880038727DF47F4B12BED67D017F4C12BED671
:107D98007DF47F4D12BED67D017F4E12BED67DF496
:107DA8007F4912BED67D017F4A12BED67DF47F4739
:107DB80012BED67D017F4812BED67D707F1312BEDB
:107DC800D67D307F1412BED67D6D7F1512BED67D4E
:107DD800707F1612BED67D707F1712BED67D307F9B
:107DE8001812BED67D6D7F1912BED67D707F1A120D
:107DF800BED68056204753303850E4F53CE53C2445
:107E080049FFE434ECFE7B007A00793E12C2B6E505
:107E18003C2447FFAD3E12BED6053CE53CC3940862
:107E280040DBE4F53CE53C2415FFE434ECFE7B0044
:107E38007A00793E12C2B6E53C2413FFAD3E12BE6D
:107E4800D6053CE53CC3940840DB7D017F0912BEA2
:107E5800D612C30B12BD9312C30B12BC0C12C30B68
:107E680012B72A12C30B12A9D612C30B12B79AC2A1
:107E780038304F39E4FD7FFF12BED6E4FDFF12BE55
:107E8800D6E4FD7F0112BED6E4FD7F0212BED6E421
:107E9800FD7F0312BED67DFE7F0612BED6E4FD7FAF
:107EA8000712BED6E4FD7F0812BED6C24F7B017A08
:107EB80001793B7F067EEF12C2B690013BE0FFF4EA
:107EC8006003EF702F7F0612BE02EF60087F061274
:107ED800BE02BFFF1590013B74FEF0FD7F0612BE87
:107EE800D67D067CEFE4FF02C0C87F0612BE029072
:047EF800013BEFF06B
:017EFC002263
:1097E500900044E06403900050706AE07D00FC90B6
:1097F500004FE0F97E002DFBEE3CFA900052E07F31
:1098050000FEEF2BFFEA3EFE900051E07A002F7834
:1098150078F6EA3E18F6E6A2E713FE08E61318A660
:109825000608F6E97E002DFFEE3CFE18E6FC08E68C
:10983500FDC3EF9D7872F6EE9C18F6A3E0FEC3ED2E
:109845009400FFEC9EFE900051E07C002F18F6EC92
:109855003E18F68027E0FE90004FE07C002400785B
:1098650078F6EC3E18F6900039E0FF78717600083E
:10987500A607A3E0FF786F760008A607D249204D1A
:109885000330530990002AE06003029936900041A5
:10989500E0FB64017037900050E0FE90004FE07CE3
:1098A5000024007878F6EC3E18F690003EE0FF7E46
:1098B500007D0A12566D7871A60608A60790003D30
:1098C500E0FF7E0012566D786FA606805FEB705F35
:1098D50090003FE0FF7E007C007D0A12566DAA06CF
:1098E500AB07A3E0F9FF7E0012566DEF2B7878F6F3
:1098F500EE3A18F6E6A2E713FE08E61318A60608E0
:10990500F6AF01E412C05FC3EF787896FFEE1896C4
:109915007871F608A60790003FE0FFE4FC12C05FEF
:10992500C37878E69FFF18E69E786FF608A607C20B
:1099350049A249305101B35006A2499251D26D2234
:0CC29200AB4DAA4CA94BA84A12BC992243
:0BC05F00FDFE754D0AF54CF54BF54A4F
:10C06A008F498E488D478C46AF4DAE4CAD4BAC4A8E
:0CC07A00AB49AA48A947A84612578522E6
:04C24D007F507EC3DD
:0BC25100EF1FAC0670011E4C70F622BF
:048F78008E3C8F3D5F
:108F7C00C3E53D94B1E53C64809480500DC3E53D60
:108F8C00944FE53C648094805002D322E53D25E06B
:108F9C00FFE53C33FE90003BE0FB75F0C4906B5B4F
:108FAC00125877E5822FF582E5833EF583E493FF33
:108FBC00EDC39F5003029168E53D25E0FFE53C338E
:108FCC00FE75F0C4EB906B5C125877E5822FF5823E
:108FDC00E5833EF583E493FFEDD39F400302916854
:108FEC00E53D646A453C6008E53D646B453C700DAD
:108FFC00900027E07007ED7002D322C322E53D6498
:10900C005C453C7024900044E0FF64026009EF640E
:10901C00046004EFB40508ED6003029166C322ED11
:10902C0064016003029166C322E53D644F453C70C8
:10903C002520410A204807EDD39400400122BD02AF
:10904C000B90014EE0C394035002C322ED70053027
:10905C005902C322D322E53D6451453C704A90002D
:10906C002DE0FF64036005EF6405702CBD0305ED76
:10907C0064056024E4FCAF040C74742FF582E434B2
:10908C0000F583E0B402031C8006ECC3940740E6B1
:10909C00ECC394075002C32290002BE0B40107EDFF
:1090AC0064016002C322D322E53D6452453C703C0E
:1090BC0090002EE0FF64036005EF6405702CBD0387
:1090CC0005ED64056024E4FCAF040C74742FF58288
:1090DC00E43400F583E0B403031C8006ECC394076E
:1090EC0040E6ECC394075002C322D322E53D6477DB
:1090FC00453C7032900045E0FF6401701FEF640244
:10910C00701AED64046005ED6002C322EDC3940493
:10911C00500A90003CE0FFED9F400122900053E08C
:10912C00900132F08034E53D6459453C702290004A
:10913C003AE0FF900039E02FFFE433CF240ACF341C
:10914C0000FEEDC39FEE6480F8748098500CC3222F
:0D915C00E53D6475453C7002C322D322C37B
:0191690022E3
:07BF9100E6FE08E6FFE4FDF7
:10BF9800EFA805088005CEC313CE13D8F9FF90018A
:10BFA80042EEF0A3EFF07E005401FF900142EEF064
:05BFB800A3EFF024FFDF
:01BFBD002261
:06B807008B468A478948C8
:10B80D00900140E4F0A304F0AF05900140E0FEA3E9
:10B81D00E0A807088005C333CE33CED8F9F0EE90FB
:10B82D000140F0306416AB46AA47A948125720FFD5
:10B83D00900140E045F0FEA3E04F8023900140E0F1
:10B84D00FEA3E0F4FFEEF4FE900140F0A3EFF0ABA9
:10B85D0046AA47A948125720FDE5F05EFEED5FFFB1
:06B86D00EE8FF012574BB4
:01B8730022B2
:10892600783C7C007D007BFF7A7079457E007F076E
:1089360012561CE4FC743C2CF8760174612CF5820A
:10894600E43400F583E0FF1258838A950089A80174
:1089560089C30289D70389F2048A06058A23068A0F
:1089660023078A23088A23098A230A8A230B8A2350
:108976000C8A7F0D8A700E8A9E0F8A9E108A9E111F
:108986008A9E128A9E138A34148A48158A5C168A2D
:10899600B5178AC7188AD2198AD71A8B051B000001
:1089A6008B27743C2CF8E6FE304104A22A8002A2F2
:1089B60028E4335EF6204303028B278055743C2C53
:1089C600F8E6FEA229E4335EF6204303028B2780F5
:1089D60041743C2CF8E6FE304104A2288002A22A0B
:1089E600E4335EF6204303028B278026743C2CF882
:1089F600E6FEA22BE4335EF6204303028B278012A9
:108A0600743C2CF8E6FEA22CE4335EF62043030207
:108A16008B27743C2CF8E66401F6028B27EF24FAC8
:108A2600FF9000FEE06F6003028B27028B2190000F
:108A3600FEE0FF64016008EF64076003028B270213
:108A46008B219000FEE0FF64026008EF640860037B
:108A5600028B27028B219000FEE0FF64036008EF83
:108A660064096003028B27028B21787B12BF914039
:108A7600047F0180117F00800D787D12BF91400434
:108A86007F0180027F00743C2CF8A607028B2774B6
:108A96003C2CF87601028B2774612CF582E43400B5
:108AA600F583E024F1FF90002AE06F7074806C90EB
:108AB60000FEE0FFC394014068EFD3940350628048
:108AC6005A9000FEE0C394074057804F304D5280C5
:108AD6004A9000FEE0FF64016004EFB40702803BA9
:108AE6009000FEE0FF64026004EFB40802802C9060
:108AF60000FEE0FF64036005EF64097024801C90AB
:108B060000FEE0FF64026004EFB40802800D9000EE
:108B1600FEE0FF64036004EFB40906743C2CF8E43D
:108B2600F60CEC6407600302893BE53C24FF9218CF
:108B3600E53D24FF9219E53E24FF921AE53F24FF06
:108B4600921BE54024FF921CE54124FF921DE5425D
:108B560024FF921F90002AE0700AD21AD219D21866
:048B6600D21DD21C2E
:018B6A0022E8
:10B874007F0112BE02EF7F00FEC006C007E412BEC5
:10B8840002EFFDD0E02DFFD0E03400FEE4FCFDC06B
:10B8940004C005C006C0077F0212BE02E4FCFDFE20
:10B8A400FBFA7901F8125785D003D002D001D000F9
:10B8B40012576AC004C005C006C0077F0312BE0247
:10B8C400E4FCFDFEFBFAF97801125785D003D0029F
:07B8D400D001D00012576AF9
:01B8DB00224A
:109D1600C2607B017A0079877D0212C10C500A90DD
:109D26000089E024FF92618006D2B2A2B2926190CD
:109D36000080E0FF64036004EFB4041790000DE0B8
:109D46007004A3E064017004D2608002C2609000D7
:109D560080802290007FE0FF64036004EFB4041863
:109D660090000BE07004A3E064017004D2608002EE
:109D7600C26090007FE0801D900081E0FF64036078
:109D860004EFB4040F306104D2608002C260788FA1
:109D9600A6078004E4788FF6A260304B01B3500426
:109DA60005528009E552D3940040021552E552C38C
:109DB600940A5003029E45E4F55230600543570865
:109DC60080035357F7788FE6607124FC6031047086
:109DD6006A206067C24D5357FEAD577F0912BED643
:109DE600900053E0900132F0E490002AF090005386
:109DF600F0FD7F7712BED6C253E4787AF6803C3007
:109E06006019C24D5357FEE490002AF0C253787A87
:109E1600F6900053E0900132F0800BD24D4357018B
:109E260090002A7404F0AD577F0912BED690002A1E
:0F9E3600E0FD900053F07F7712BED6A260924BF2
:019E450022FA
:1094EF007F0712BE028F307FE87E0312C251E53034
:1094FF006009647D6005E530F4703412A18A9248EA
:10950F0012B94492413048089000D67404F0801389
:10951F009000D630410A7402F090002714F08003B7
:10952F007401F09000D6E0FD7F0712BED680069042
:10953F0000D6E530F07F0812BE029000D6E0FED3D1
:10954F0094035067EF24FE24FD501724047048EE57
:10955F00B40208D2419000277401F09000227401E8
:10956F0080459000227401F0D250EFC39404400262
:10957F00D23BEEB40303D24822EEB4020FD248908E
:10958F0000277403F0439B30E4F5A322EE640160DF
:10959F0003029679D24822EEB40208D241900027F6
:1095AF007401F0E4900022F0C250229000D6E0FE49
:1095BF0064046008EE640C600302965ED248EEB459
:1095CF000C0ED24C9000277402F0439BC0E4F5A31D
:1095DF00EFD3940040089000227401F08005E490CE
:1095EF000022F0EFD39401400EEF64046009EF64A2
:1095FF00066004D2438002C243EFD39401400DEFC3
:10960F00647D6008EFF46004D2508002C250EFC353
:10961F0094084015EF647D6010EFF4600CC2A7C290
:10962F00A6C293C290C291C2949000D6E0B4040D2A
:10963F00BF050AC2A7C2A6C293C290C291EFC3943C
:10964F000A4027EF647D6022EFF4601ED23B229028
:10965F0000D6E0B40D14D2489000277404F0D24124
:0A966F009000227401F0C250D23BBB
:0196790022CE
:08C172007D01E4FF12C17A0F08
:0EC17A00EDBF010524FF92232224FF92242210
:03002B0002A55FCC
:10A55F00C0E0C0F0C083C082C0D075D000C000C0C2
:10A56F0001C002C003C004C005C006C007C2CF901F
:10A57F000002125809EF2401FFE43EFEE43DFDE422
:10A58F003CFC90000212582130463190004CE0FF05
:10A59F00E4FCFDFE7BE87A03F9F812578590000280
:10A5AF00125815D31257F8401312C17290000212AD
:10A5BF00584600000000C246787976007879E66444
:10A5CF0001705D7873E6FA08E6D39400EA6480942C
:10A5DF0080402AE616187001162058099000CDE425
:10A5EF0075F001803290004CE0FF7E007C037DE827
:10A5FF0012566D9000CDEEF0A3EFF08023C3EA6406
:10A60F00809480501B787406E6187001069000CD78
:10A61F0020550974FFF5F012570A8004E4F0A3F0F7
:10A62F00D007D006D005D004D003D002D001D0007F
:0BA63F00D0D0D082D083D0F0D0E03229
:10BFBE0090000212584600000000E49000CDF0A35D
:10BFCE00F0900023F0A3F07D017F0112C17A1D1FB6
:0ABFDE0012C17AD246E47879F62207
:10BC54007879E624FE603A04703A7873E6FA08E6E6
:10BC6400FBD39400EA64809480400BE4FD7F0112CE
:10BC7400C17A0D1F8010C3EA64809480500BE4FDE8
:10BC8400FF12C17A0D0F02C17A12C172E47879F6FB
:05BC94002212BFBE22D8
:10BDCB00C2AF9000021258099000CF125821D2AF87
:10BDDB007F007E5C7D267C059000CF125815D31218
:10BDEB0057F84012C2AF90000212584600000000F4
:07BDFB00D2AF787976022235
:10934200900023E0FEA3E0FF9000CAE0FCA3E0FD52
:10935200C39FFFEC9E900025F0A3EFF0D3ED945F46
:10936200EC64809480403690001FE475F00112573F
:109372000AD3900020E0945890001FE094024074B9
:10938200E4F0A3F090004CE0FF7E007C007DC81268
:10939200566D7873A60608A607D258804AC3900075
:1093A200CBE094059000CAE064809480503F900026
:1093B2001FE475F00112570AD3900020E0945890F0
:1093C200001FE09402402DE4F0A3F090004CE0FF77
:1093D200E49FFFE49400FE7C007DC812566D787312
:1093E200A60608A607D255787976018007E4900090
:1093F2001FF0A3F0900025E0FEA3E0FF12C1EAC334
:10940200EF9405EE6480948040020553C3E55364F3
:109412008094814005D245E4F5532045030294EE41
:10942200C245E4F553C255C2589000CAE0FEA3E01B
:10943200FFD39405EE648094805012900024E0944F
:1094420005900023E0648094804002D23FC3EF94F1
:109452005FEE648094804012900024E0945F90005C
:1094620023E0648094805002D24090004CE0F97571
:10947200F00AA4FFAEF07873EEF608EFF69000CA99
:10948200E0FCA3E0FD12566D7873EEF608EFF6905D
:1094920000CDE0FCA3E0FDC3EF9DF6EE9C18F63094
:1094A2003F19E9FF7E007C007DC812566DC37874B7
:1094B200E69FF618E69EF6C23FD25530401B90005A
:1094C2004CE0FF7E007C007DC812566D7874EF265A
:1094D200F618EE36F6C240D258787976019000CA74
:0D94E200E0FFA3E0900023CFF0A3EFF02205
:10C1C400E4FD7F0412BF6E12BDCB204603129342DE
:03C1D40002BC5456
:0EC25C0000113333143C3C00113333143C3CCE
:09B56B00027F323242010E0000A1
:06BE6E008B428A43894467
:10BE74007F01AE05EFA806088002C333D8FCFF306B
:10BE8400610CAB42AA43A9441256424F800D63078A
:0EBE9400FFAB42AA43A9441256425F12565B0E
:01BEA200227D
:06C106007B017A0079883C
:10C10C007F01AE05EFA806088002C333D8FCFF12EE
:05C11C0056425F24FF04
:01C1210022FB
:10BD5A00C26C90009C7403F0A304F090009B7402E0
:10BD6A00F090009E7405F09000A3741CF0A304F0F8
:10BD7A00A304F0A304F0A304F0A304F0A304F0A323
:09BD8A0004F0E4FD7F0502BF6E28
:10C0A8008B45EF7B017A01790EB50509E545240238
:10C0B800FDC2648007E5452402FDD26412B8072258
:10BF36008F4530630C74FE2FF582E43400F583E4FC
:10BF4600F07B017A01790ED264AD4512B8077B0108
:0EBF56007A01790EE5452402FDC26402B807A7
:02242E008F42DB
:10243000900038E01470030224C61470030224F4E0
:10244000147003022585147003022616147003020B
:1024500026A124056003022728E558B402030226BA
:1024600046747F2542F8E62402FFE433FE74852596
:1024700042F8E6D39FEE6480F874809840177B00A2
:102480007A00797DC264AD4212B8077B007A007988
:102490007BD264802C747F2542F8E624FEFF74858D
:1024A0002542F8E6C39F7B007A00797D5004D26410
:1024B0008002C264AD4212B8077B007A00797BC209
:1024C00064AD420227257B007A00797D304411C239
:1024D00064E4FD12B8077B007A00797BD264800F38
:1024E000D264E4FD12B8077B007A00797BC264E411
:1024F000FD0227257B017A0079877D0212C10C50ED
:102500000A900089E024FF92618006D2B2A2B292C2
:1025100061900080E0B4051490000DE07004A3E029
:1025200064017004D262802FC262802B90007FE031
:10253000B4051490000BE07004A3E064017004D2B1
:10254000628014C2628010900081E0B4050930619D
:1025500004D2628002C2627B007A00797D3062110F
:10256000C264E4FD12B8077B007A00797BD26480F4
:102570000FD264E4FD12B8077B007A00797BC26455
:10258000E4FD0227257B017A0079877D0212C10CC8
:10259000500A900089E024FF92618006D2B2A2B274
:1025A0009261900080E0B4051490000DE07004A3E7
:1025B000E064017004D262802FC262802B90007FA1
:1025C000E0B4051490000BE07004A3E06401700413
:1025D000D2628014C2628010900081E0B40509309C
:1025E0006104D2628002C2627B007A00797D20623F
:1025F00011C264E4FD12B8077B007A00797BD264D3
:10260000800FD264E4FD12B8077B007A00797BC2A8
:1026100064E4FD02272590000BE0FEA3E0FF90019B
:102620003EEEF0FCA3EFF0FD900050E0FE90004F76
:10263000E07A002400FFEA3ECF24F6CF34FFFEC349
:10264000ED9FEC9E501A7B007A00797DD264E4FD08
:1026500012B8077B007A00797BC264E4FD0227256B
:10266000900050E0FE90004FE07C002400FFEC3E24
:10267000CF240ACF3400FED390013FE09F90013E6B
:10268000E09E50030227287B007A00797DC264E433
:10269000FD12B8077B007A00797BD264E4FD022743
:1026A0002590000DE0FEA3E0FF90013EEEF0FCA3BC
:1026B000EFF0FD900050E0FE90004FE07A00240023
:1026C000FFEA3ECF24F6CF34FFFEC3ED9FEC9E50D1
:1026D000197B007A00797DD264E4FD12B8077B0093
:1026E0007A00797BC264E4FD803B900050E0FE906C
:1026F000004FE07C002400FFEC3ECF240ACF3400E2
:10270000FED390013FE09F90013EE09E401A7B0087
:102710007A00797DC264E4FD12B8077B007A007903
:102720007BD264E4FD12B807E54225E0FFE433FE06
:10273000C3742B9FFFE49EFE742B2FF58274003E22
:10274000F583E0FF702174812542F87664E54275D7
:10275000F006A42426F582E43401F583E0FE7483B8
:102760002542F8A6068063EFB4060974832542F873
:10277000E4F6803EE54225E0FFE433FEC3742B9F80
:10278000FFE49EFE742B2FF58274003EF583E0FF7C
:10279000E54275F006A42426F582E43401F583E5CC
:1027A000822FF582E43583F583E0FF74832542F8B8
:1027B000A607E54275F006A42426F582E43401F567
:1027C00083E0FF74812542F8A60774832542F974DB
:1027D000852542F8E6FFC397400A74812542F8EF49
:1027E000D3964042900044E064056044787BE6FE66
:1027F00008E6FFAD4212BF98500F74812542F9746C
:10280000852542F8E6C397401D787DE6FE08E6FF81
:10281000AD4212BF98501974832542F97485254240
:10282000F8E6D397400A746A2542F8E4F6022CB021
:10283000787DE6FE08E6FFAD4212BF984003022A0B
:1028400061E4788FF6E54225E0FFE433FEC3742CA3
:102850009FFDE49EFC742B2DF58274003CF583E013
:10286000FD788FE6FCC39D503BC3742B9FFFE49E15
:10287000FE742B2FF58274003EF583E02CFFE542B9
:1028800075F006A42426F582E43401F583E5822F51
:10289000F582E43583F583E0FF74912CF8A6077880
:1028A0008F0680A1E4788FF6E54225E0FFE433FE51
:1028B000C3742C9FFFE49EFE742B2FF58274003EA0
:1028C000F583E0FFC374069FFE788FE6FDC39E503C
:1028D0000CEF2D2491F87602788F0680CB74852535
:1028E00042F8E6FFD39403500B788FA60774852532
:1028F00042F876037896E624FEFF74852542F8E6D2
:10290000FEC39F5009746A2542F87606804BEED3C9
:102910007891964009746A2542F8E4F6803BE478A1
:1029200090F67890E6FFC39404502E74922FF974B9
:10293000852542F8E6FFD397401A7890E6FE249169
:10294000F8E624FEFDEFC39D500AEE04FF746A25ED
:1029500042F8A60778900680C97891E6FF24FEFE2B
:1029600074852542F8E6FDC39E4015EDD39F5010B7
:10297000746A2542F8E6FF64016005EF60027601A3
:102980007892E6FF24FEFE74852542F8E6FDC39E9C
:102990004017EDD39F5012746A2542F8E6FF640198
:1029A0006007EF6402600276027893E6FF24FEFE81
:1029B00074852542F8E6FDC39E4017EDD39F501263
:1029C000746A2542F8E6FF64026007EF6403600260
:1029D00076037894E6FF24FEFE74852542F8E6FD32
:1029E000C39E4017EDD39F5012746A2542F8E6FF4C
:1029F00064036007EF6404600276047895E6FF24C0
:102A0000FEFE74852542F8E6FDC39E4017EDD39F78
:102A10005012746A2542F8E6FF64046007EF64050B
:102A2000600276057896E6FF24FEFE74852542F85E
:102A3000E6FDC39E4017EDD39F5012746A2542F8FD
:102A4000E6FF64056007EF6406600276067485257C
:102A500042F8E6B4030B788FE6FF74852542F8A6AA
:102A600007787BE6FE08E6FFAD4212BF98400302FE
:102A70002CB0E4788FF6E54225E0FFE433FEC37422
:102A80002B9FFFE49EFE742B2FF58274003EF5838E
:102A9000E0FF788FE6C39F5028E6FFE54275F00619
:102AA000A42426F582E43401F583E5822FF582E43F
:102AB0003583F583E0FE74912FF8A606788F0680A3
:102AC000B5E4788FF6E54225E0FFE433FEC3742BCE
:102AD0009FFFE49EFE742B2FF58274003EF583E089
:102AE000FFC374069FFE788FE6FDC39E500CEF2D4A
:102AF0002491F87666788F0680CB7896E62402FFDC
:102B0000E433FE74852542F8E6FDD39FEE6480F839
:102B10007480984009746A2542F8760C8056EDC39B
:102B20007891965009746A2542F8E4F68046E47874
:102B300090F67890E6FFC39404503974922FF9749C
:102B4000852542F8E6FFC39750257890E6FE24914C
:102B5000F8E62402FDE433FCEFD39DEC6480F874C6
:102B60008098400BEE2407FF746A2542F8A6077888
:102B7000900680BE74852542F8E6FF7891E6FEEF68
:102B8000C39E4023EE2402FDE433FCD3EF9DEC64AE
:102B900080F87480985010746A2542F8E6FF640744
:102BA0006005EF6002760774852542F8E6FF7892AB
:102BB000E6FEEFC39E4025EE2402FDE433FCD3EF96
:102BC0009DEC6480F87480985012746A2542F8E68F
:102BD000FF64076007EF6408600276087485254289
:102BE000F8E6FF7893E6FEEFC39E4025EE2402FD53
:102BF000E433FCD3EF9DEC6480F874809850127439
:102C00006A2542F8E6FF64086007EF64096002760F
:102C10000974852542F8E6FF7894E6FEEFC39E40EE
:102C200025EE2402FDE433FCD3EF9DEC6480F874C0
:102C300080985012746A2542F8E6FF64096007EF35
:102C4000640A6002760A74852542F8E6FF7895E604
:102C5000FEEFC39E4025EE2402FDE433FCD3EF9D3E
:102C6000EC6480F87480985012746A2542F8E6FF8C
:102C7000640A6007EF640B6002760B74852542F8E6
:102C8000E6FF7896E6FEEFC39E4025EE2402FDE4C3
:102C900033FCD3EF9DEC6480F87480985012746A12
:102CA0002542F8E6FF640B6007EF640C6002760CC7
:102CB00074FE2542F582E43400F583E0FF74432579
:102CC00042F8A60790010EE0FEA3E0FFAD4212BF5E
:102CD000984003022D5A900018E0FEA3E0FFAD4299
:102CE00012BF98407574FE2542F582E43400F583E6
:102CF000E0704C746A2542F8E6D39406401F9001B8
:102D000000E0FEA3E0FFAD4212BF98401074FE2524
:102D100042F582E43400F5837407F08030746A254C
:102D200042F8E6FFD394004024EF9407501F90012F
:102D300002E0FEA3E0FFAD4212BF98401080007495
:102D4000FE2542F582E43400F583E004F07B017A4D
:102D500001790EC264AD4212B80790010EE0FEA3E5
:102D6000E0FFE5422402FD12BF98504F900018E0AA
:102D7000FEA3E0FFAD4212BF98404074FE2542F52D
:102D800082E43400F583E0FFB4070F74FE2542F5BA
:102D900082E43400F583E4F08011EF600E74FE25C8
:102DA00042F582E43400F583E014F07B017A017986
:102DB0000EE5422402FDC26412B807746A2542F887
:102DC000E61258832DEC012E2D022E7E032ED10407
:102DD0002F27052F7D062FC8072FFD083047093004
:102DE000980A30EA0B313E0C0000319074FE254207
:102DF000F582E43400F583E0FFD394005003023001
:102E000093EF940740030230937B017A01790EC25D
:102E100064AD4212B80774FE2542F582E43400F531
:102E200083E0FFAB427D0102311902309374FE252D
:102E300042F582E43400F583E0FFD394014026EFAD
:102E4000940750217B017A01790EC264AD4212B819
:102E50000774FE2542F582E43400F583E0FFAB42BF
:102E60007D0202311974FE2542F582E43400F583B7
:102E7000E0B40105C263023189D26302318974FE74
:102E80002542F582E43400F583E0FFD39402402626
:102E9000EF940750217B017A01790EC264AD421292
:102EA000B80774FE2542F582E43400F583E0FFABF9
:102EB000427D0302311974FE2542F582E43400F5A7
:102EC00083E0FF6402605AEFB4010302308E0230E7
:102ED0009374FE2542F582E43400F583E0FFD39439
:102EE000034026EF940750217B017A01790EC264DA
:102EF000AD4212B80774FE2542F582E43400F58332
:102F0000E0FFAB427D0402311974FE2542F582E4F4
:102F10003400F583E0FFC394034009EFD3940150DC
:102F20000302308E02309374FE2542F582E43400B1
:102F3000F583E0FFD394044026EF940750217B01F2
:102F40007A01790EC264AD4212B80774FE2542F5CB
:102F500082E43400F583E0FFAB427D050231197451
:102F6000FE2542F582E43400F583E0FFD39404505B
:102F700009EFC39401400302308E02309374FE25A2
:102F800042F582E43400F583E0B4061E7B017A0149
:102F9000790EC264AD4212B80774FE2542F582E490
:102FA0003400F5837406F00231E174FE2542F582A7
:102FB000E43400F583E0FFD394055009EFC3940196
:102FC000400302308E02309374FE2542F582E434D1
:102FD00000F583E0D3940640217B017A01790EC28B
:102FE00064AD4212B80774FE2542F582E43400F560
:102FF00083E0FFAB427D0702311902309374FE2556
:1030000042F582E43400F583E0D3940740217B014C
:103010007A01790EC264AD4212B80774FE2542F5FA
:1030200082E43400F583E0FFAB427D08023119747D
:10303000FE2542F582E43400F583E0B40704C26360
:103040008002D26302318974FE2542F582E43400A5
:10305000F583E0D3940840217B017A01790EC264A4
:10306000AD4212B80774FE2542F582E43400F583C0
:10307000E0FFAB427D0902311974FE2542F582E47E
:103080003400F583E0FF64086004EFB40705C26311
:10309000023189D26302318974FE2542F582E4341B
:1030A00000F583E0D3940940207B017A01790EC2B8
:1030B00064AD4212B80774FE2542F582E43400F58F
:1030C00083E0FFAB427D0A805074FE2542F582E426
:1030D0003400F583E0FFD394094005EF94074005E1
:1030E000C263023189D26302318974FE2542F582BE
:1030F000E43400F583E0D3940A40247B017A01791B
:103100000EC264AD4212B80774FE2542F582E43463
:1031100000F583E0FFAB427D0B12C0A80231E174E1
:10312000FE2542F582E43400F583E0FFD3940A40A3
:1031300005EF94074004C263804FD263804B74FE56
:103140002542F582E43400F583E0D3940B401D7BE7
:10315000017A01790EC264AD4212B80774FE2542AD
:10316000F582E43400F583740CF0807574FE25421A
:10317000F582E43400F583E0FFD3940B4005EF942F
:10318000074004C2638002D263AF4212BF3680514F
:103190007B017A01790EC264AD4212B80774FE2534
:1031A00042F582E43400F583E0C39401400F7B01D3
:1031B0007A01790EE5422402FDD2648021746A25E9
:1031C00042F8E6FF74FE2542F582E43400F583EF11
:1031D000F07B017A01790EE5422402FDC26412B847
:1031E0000774FE2542F582E43400F583E0FF744362
:1031F0002542F8E66F60147B017A007918D264AD3D
:103200004212B807E4FD7F0F12BF6E9000FEE0602F
:10321000030232BFE543D394004051E54394075085
:103220004B7F5712BE02EF601E7B017A017902D2FA
:1032300064E4FD12B8077F5712BE0290010CEFF054
:10324000E4FD7F1012BF6E7F5812BE02EF60707BEC
:10325000017A017900D264E4FD12B8077F5812BEEA
:103260000290010AEFF0E4FD7F118050E543C39422
:1032700007404C7F5712BE02EF601E7B017A017936
:1032800000D264E4FD12B8077F5712BE0290010A13
:10329000EFF0E4FD7F1112BF6E7F5812BE02EF60A7
:1032A0001E7B017A017902D264E4FD12B8077F58CF
:1032B00012BE0290010CEFF0E4FD7F1012BF6E20F1
:1032C0006C29E490010EF0A3F0900102F0A3F090BD
:1032D0000100F0A3F0746A2542F8E6FF74FE25426F
:0B32E000F582E43400F583EFF0D26CBF
:0132EB0022C0
:10028C00E4FD7F0212BF6E1297E5E4F53CAF3C1221
:10029C00242E053CE53CC3940240F2305D1E9000D8
:1002AC0056E09000FEF090007EE0FF7E007C007D2A
:1002BC003C12566D900110EEF0A3EFF09000FEE0B2
:1002CC00FFD3940690002AE075F0075008A424B1DF
:1002DC00FEEF2E8017A424B1FF9000FEE02FFF90BC
:1002EC000057E0FEC374069EFEC3EF9EFF12BE02D3
:1002FC00900106E4F0A3EFF09000FFE0FFD394062A
:10030C00501390002AE07005EF24B1802F9000FF6D
:10031C00E024D4802790002AE0900055700FE0FF75
:10032C00C374069FFF9000FFE024B1800DE0FFC373
:10033C0074069FFF9000FFE024D4C39FFF12BE02FF
:10034C00900108E4F0A3EFF0E4F53C7468253CF56B
:10035C0082E43400F583E0FFB4020F7985E7D378AB
:10036C008696741240208011801CEFB40326798588
:10037C00E7C37886967412500D253CF582E434015F
:10038C00F583E4F08028253CF582E43401F5837490
:10039C0001F0801A7468253CF582E43400F583E0A2
:1003AC00FF7412253CF582E43401F583EFF07412EE
:1003BC00253CF582E43401F583E025E02406F58242
:1003CC00E43401F583E0FEA3E0FFAD3C12BF98924C
:1003DC00647B017A017904AD3C12B807053CE53C1D
:1003EC00C394055003020357900072E0700890010B
:1003FC0005E0F5248012900104A3E0FF139220EF96
:10040C00A2E19221A2E29222E4F53CE53C2491FF88
:10041C0012BE02BF020F7985E7D3788696746D40C1
:10042C002780188023E53C2491FF12BE02BF0324D1
:10043C007985E7C3788696746D500D253CF582E47A
:10044C003400F583E4F0800C253CF582E43400F5AF
:10045C00837401F0053CE53CC3940240AEE558249E
:10046C00FE70030205702402600302060C90006DFE
:10047C00E0FF25E0248CF8743226F618E436F6EF0B
:10048C0025E0248CF9D3E794E819E7648094834041
:10049C000AE025E0248BF8E4F608F690006EE0FF05
:1004AC0025E02488F874CE26F61874FF36F6EF256E
:1004BC00E02488F9C319E764809480500BE025E0B0
:1004CC002487F876030876E890014EE0C394034045
:1004DC003A303B3790006DE025E0248BF8E6FE08BF
:1004EC00E6FFD394EEEE64809482400790002B7468
:1004FC00028038D3EF9490EE648094814007900092
:10050C002B74018004E490002B802090006DE0257A
:10051C00E0248CF9D3E794F419E7648094814007C4
:10052C0090002B74018004E490002BF0900119745E
:10053C0005F0788BE6FE08E6FF7C007D041256D4AD
:10054C008F3CAD3C7F0A12BED67F0A12BE02EF650D
:10055C003C70030212AD7B9D7D9D7F0D12C28B12F0
:10056C00C30B80F290003BE064017047E55624C059
:10057C00FFE55534FEFE7C007D0512566D7D09129B
:10058C0056D4788BA60608A607900050E0FE900083
:10059C004FE07C002400FFEC3ECF24C0CF34FEFEA5
:1005AC007D0512566D7D0912567F7887A60608A622
:1005BC0007801B788BA65508A656900050E0FE903D
:1005CC00004FE07C0024007888F6EC3E18F6D378D7
:1005DC008CE694E818E664809483400576030876EC
:1005EC00E8D37888E694E818E6648094834005762E
:1005FC00030876E85324F8A253724D92200212ADF0
:10060C009000FEE0FFD394065005EF24DB8012909F
:10061C000057E0FFC374069FFF9000FEE024DBC38D
:10062C009FFF12BE028F3D9000FFE0FFD394065057
:10063C0005EF24E28012900055E0FFC374069FFF83
:10064C009000FFE024E2C39FFF12BE028F3E900099
:10065C006DE0FF243DF8E6540314700302087D148A
:10066C0060101470030207772403600302088302EE
:10067C00087674832FF8E6FE74852FF8E6F9C39E8E
:10068C00400302077490006DE0FD25E0FFE433FEAB
:10069C00C3742B9FFFE49EFE742B2FF58274003ED7
:1006AC00F583E0FF74FE2DF582E43400F583E0FE63
:1006BC00EF2EFF90006DE075F006A42425F582E482
:1006CC003401F583E5822FF582E43583F583E0FF71
:1006DC00E9FDC3EF9DFFE49400FEE4FCFD754DE8DD
:1006EC00754C03F54BF54A12C06AC004C005C00630
:1006FC00C00790006DE0FD25E0FFE433FEC3742BD2
:10070C009FFBE49EFA742B2BF58274003AF583E080
:10071C00FCC3742C9FFFE49EFE742B2FF582740097
:10072C003EF583E02CFFED75F006A42425F582E45C
:10073C003401F583E5822FF582E43583F583E0FF00
:10074C00E4F8F9FAAB07D007D006D005D00412BCF8
:10075C00998E408F41D3E54194E8E54064809483C1
:10076C00500302088302087D02087690006DE0FFBA
:10077C002483F8E6FE74852FF8E6F9C39E40030245
:10078C000876E0FD25E0FFE433FEC3742B9FFFE405
:10079C009EFE742B2FF58274003EF583E0FF74FEF1
:1007AC002DF582E43400F583E0FEEF2EFF90006D12
:1007BC00E075F006A42425F582E43401F583E58286
:1007CC002FF582E43583F583E0FFE9FDC3EF9DFF50
:1007DC00E49400FEE4FCFD754DF4754C01F54BF50D
:1007EC004A12C06AC004C005C006C00790006DE084
:1007FC00FD25E0FFE433FEC3742B9FFBE49EFA74EB
:10080C002B2BF58274003AF583E0FCC3742C9FFF0C
:10081C00E49EFE742B2FF58274003EF583E02CFFD2
:10082C00ED75F006A42425F582E43401F583E58208
:10083C002FF582E43583F583E0FFE4F8F9FAAB0792
:10084C00D007D006D005D00412BC998E408F4174CD
:10085C00F42541F54174013540F540D3E54194E868
:10086C00E54064809483400F8007E4F540F54180B7
:10087C00067540037541E890006DE0243DF8E620D4
:10088C00E603020963E0FD25E0FFE433FEC3742BAD
:10089C009FFFE49EFE742B2FF58274003EF583E0DF
:1008AC00FF74FE2DF582E43400F583E0FEEF2EFF9D
:1008BC0090006DE0FE75F006A42425F582E4340169
:1008CC00F583E5822FF582E43583F583E0FD7485AD
:1008DC002EF8E6FFC3ED9FFFE49400FEE4FCFD75EB
:1008EC004DF4754C01F54BF54A12C06AC004C005B5
:1008FC00C006C00790006DE0FD25E0FFE433FEC3A9
:10090C00742B9FFBE49EFA742B2BF58274003AF542
:10091C0083E0FCC3742C9FFFE49EFE742B2FF582A6
:10092C0074003EF583E02CFFED75F006A42425F54C
:10093C0082E43401F583E5822FF582E43583F58377
:10094C00E0FFE4F8F9FAAB07D007D006D005D004E5
:10095C0012BC998E408F41D3E54194E8E540648008
:10096C00948340067540037541E8900046E0FBB463
:10097C00020DAE40AF417C007D021256D4805CEB80
:10098C0064037045AE40AF41FC7D0512566D0D12EF
:10099C0056D4EF24B1FFE43EFE90006DE0FD25E05F
:1009AC00248BF8A60608A607ED25E0248BF8E6FEB6
:1009BC0008E6D394E8EE64809483403DED25E02472
:1009CC008BF876030876E88030900046E0B4041B80
:1009DC00C374E89541FF74039540FE90006DE025CB
:1009EC00E0248BF8A60608A607800E90006DE02583
:1009FC00E0248BF8A64008A64190006EE0FF243D51
:100A0C00F8E6FE13135403147003020DC91460109E
:100A1C00147003020BEE24036003020DCF020DC20F
:100A2C0074812FF8E6FE74852FF8E6FFD39E5003F1
:100A3C00020AF490006EE0FE24FEF582E43400F528
:100A4C0083E0FDEE75F006A4241FF582E43401F575
:100A5C0083E5822DF582E43583F583E0FDC3EF9DBC
:100A6C00FFE49400FEE4FCFD754DE8754C03F54B7A
:100A7C00F54A12C06AC004C005C006C00790006EDB
:100A8C00E0FD25E0FFE433FEC3742B9FFFE49EFEE4
:100A9C00742B2FF58274003EF583E0FFED75F006A4
:100AAC00A42425F582E43401F583E5822FF582E454
:100ABC003583F583E0FFC374649FFFE49400FEE488
:100ACC00F8F9AA06AB07D007D006D005D00412BCA3
:100ADC00998E408F41D3E54194E8E540648094833E
:100AEC005003020DCF020DC990006EE0FF2483F875
:100AFC00E6FE74852FF8E6F9C39E4003020BEBE08B
:100B0C00FD25E0FFE433FEC3742B9FFFE49EFE74CF
:100B1C002B2FF58274003EF583E0FF74FE2DF582D9
:100B2C00E43400F583E0FEEF2EFF90006EE075F0EC
:100B3C0006A42425F582E43401F583E5822FF582A1
:100B4C00E43583F583E0FFE9FDC3EF9DFFE49400FA
:100B5C00FEE4FCFD754DE8754C03F54BF54A12C0EF
:100B6C006AC004C005C006C00790006EE0FD25E019
:100B7C00FFE433FEC3742B9FFBE49EFA742B2BF51E
:100B8C008274003AF583E0FCC3742C9FFFE49EFE54
:100B9C00742B2FF58274003EF583E02CFFED75F07D
:100BAC0006A42425F582E43401F583E5822FF58231
:100BBC00E43583F583E0FFE4F8F9FAAB07D007D00E
:100BCC0006D005D00412BC998E408F41D3E54194D8
:100BDC00E8E540648094835003020DCF020DC902F6
:100BEC000DC290006EE0FF2481F8E6FE74852FF8AC
:100BFC00E6FFD39E5003020CC3E0FE24FEF582E414
:100C0C003400F583E0FDEE75F006A4241FF582E4B4
:100C1C003401F583E5822DF582E43583F583E0FD1F
:100C2C00C3EF9DFFE49400FEE4FCFD754DF4754CA0
:100C3C0001F54BF54A12C06AC004C005C006C007D6
:100C4C0090006EE0FD25E0FFE433FEC3742B9FFFA4
:100C5C00E49EFE742B2FF58274003EF583E0FFEDCD
:100C6C0075F006A42425F582E43401F583E5822F82
:100C7C00F582E43583F583E0FFC374649FFFE4944D
:100C8C0000FEE4F8F9AA06AB07D007D006D005D0D1
:100C9C000412BC998E408F4174F42541F5417401C6
:100CAC003540F540D3E54194E8E5406480948350A9
:100CBC0003020DCF020DC990006EE0FF2483F8E60D
:100CCC00FE74852FF8E6F9C39E4003020DC2E0FDC9
:100CDC0025E0FFE433FEC3742B9FFFE49EFE742BD0
:100CEC002FF58274003EF583E0FF74FE2DF582E44F
:100CFC003400F583E0FEEF2EFF90006EE075F006F9
:100D0C00A42425F582E43401F583E5822FF582E4F1
:100D1C003583F583E0FFE9FDC3EF9DFFE49400FE0E
:100D2C00E4FCFD754DF4754C01F54BF54A12C06AA7
:100D3C00C004C005C006C00790006EE0FD25E0FFB2
:100D4C00E433FEC3742B9FFBE49EFA742B2BF582C9
:100D5C0074003AF583E0FCC3742C9FFFE49EFE7490
:100D6C002B2FF58274003EF583E02CFFED75F00619
:100D7C00A42425F582E43401F583E5822FF582E481
:100D8C003583F583E0FFE4F8F9FAAB07D007D0061A
:100D9C00D005D00412BC998E408F4174F42541F5D6
:100DAC004174013540F540D3E54194E8E540648059
:100DBC009483400F8007E4F540F5418006754003AD
:100DCC007541E890006EE0FF243DF8E620E7030251
:100DDC000E81E0FE24FEF582E43400F583E0FDEEA6
:100DEC0075F006A4241FF582E43401F583E5822D09
:100DFC00F582E43583F583E0FD74852FF8E6C39D19
:100E0C00FFE49400FEE4FCFD754DF4754C01F54BCC
:100E1C00F54A12C06AC004C005C006C00790006E37
:100E2C00E0FD25E0FFE433FEC3742B9FFFE49EFE40
:100E3C00742B2FF58274003EF583E0FFED75F00600
:100E4C00A42425F582E43401F583E5822FF582E4B0
:100E5C003583F583E0FFC374649FFFE49400FEE4E4
:100E6C00F8F9AA06AB07D007D006D005D00412BCFF
:100E7C00998E408F41D3E54194E8E540648094839A
:100E8C0040067540037541E8900047E0FBB4020D45
:100E9C00AE40AF417C007D021256D4805CEB640303
:100EAC007045AE40AF41FC7D0512566D0D1256D407
:100EBC00EF24B1FFE43EFE90006EE0FD25E02487B8
:100ECC00F8A60608A607ED25E02487F8E6FE08E656
:100EDC00D394E8EE64809483403DED25E02487F8BC
:100EEC0076030876E88030900047E0B4041BC374A6
:100EFC00E89541FF74039540FE90006EE025E024D8
:100F0C0087F8A60608A607800E90006EE025E02460
:100F1C0087F8A64008A6417D0512C10650287FFB24
:100F2C0012BE02EF7F00FEC006C0077FFA12BE029F
:100F3C00EFFDD0E02DFFD0E03400FE788BF608EF0B
:100F4C00F608A60608F67D0612C10650287FF9128F
:100F5C00BE02EF7F00FEC006C0077FF812BE02EF94
:100F6C00FDD0E02DFFD0E03400FE7887F608EFF6D8
:100F7C0008A60608F6900072E0640160030212AD48
:100F8C0090006DE0FF243DF8E6C454031470030296
:100F9C0012751460101470030210E724036003022E
:100FAC00127E02126C74812FF8E6FB74852FF8E622
:100FBC00FDD39B406790006DE025E0FFE433FEC35A
:100FCC00742B9FFFE49EFE742B2FF58274003EF56C
:100FDC0083E0B4010302111B90006DE075F006A4D0
:100FEC002427F582E43401F583E0C39B70030212DD
:100FFC007E90006DE0FF2481F8E6FD74852FF8C328
:10100C00E69D75F064A4FFAEF0E075F006A424270D
:10101C00F582E43401F583E0C302113390006DE0F6
:10102C00FF2483F8E6FE74852FF8E6FDC39E40038B
:10103C000210E4E0FB25E0FFE433FEC3742C9FFFB9
:10104C00E49EFE742B2FF58274003EF583E0B40110
:10105C00030211BB90006DE0FD25E0FFE433FEC3FD
:10106C00742B9FFFE49EFE742B2FF58274003EF5CB
:10107C0083E0FFED75F006A42427F582E43401F536
:10108C0083E5822FF582E43583F583E0FE74832BB0
:10109C00F8C3E69E700302127E90006DE075F006B8
:1010AC00A42427F582E43401F583E5822FF582E44C
:1010BC003583F583E0FF90006DE0FB2483F8E6FABE
:1010CC00C39FFDE49400FC74852BF8C3EA9675F07D
:1010DC0064A4FFAEF00211D102126C90006DE0FF1F
:1010EC002481F8E6FB74852FF8E6FDD39B500302B0
:1010FC001186E025E0FFE433FEC3742B9FFFE49ED2
:10110C00FE742B2FF58274003EF583E0B401219020
:10111C00006DE02481F8E6FCC3ED9C75F064A4FF3F
:10112C00AEF0ECFDC374649DFDE49400FC0211D19F
:10113C0090006DE075F006A42427F582E43401F5E7
:10114C0083E0C39B700302127E90006DE0FF24814C
:10115C00F8E6FD74852FF8C3E69D75F064A4FFAE28
:10116C00F0E075F006A42427F582E43401F583E061
:10117C00C39DFDE49400FC02125990006DE0FF2425
:10118C0083F8E6FE74852FF8E6FDC39E4003021239
:10119C006CE0FB25E0FFE433FEC3742C9FFFE49E60
:1011AC00FE742B2FF58274003EF583E0B401209081
:1011BC00006DE02483F8E6FCC39D75F064A4FFAEDB
:1011CC00F0ECFD7C001256D49000CAEE0212669030
:1011DC00006DE0FD25E0FFE433FEC3742B9FFFE4BC
:1011EC009EFE742B2FF58274003EF583E0FFED75A7
:1011FC00F006A42427F582E43401F583E5822FF56B
:10120C0082E43583F583E0FE74832BF8C3E69E609D
:10121C006190006DE075F006A42427F582E434019A
:10122C00F583E5822FF582E43583F583E0FF9000AA
:10123C006DE0FB2483F8E6FAC39FFDE49400FC7494
:10124C00852BF8C3EA9675F064A4FFAEF01256D461
:10125C00EF249CFFEE34FF9000CAF0A3EFF0801255
:10126C00E49000CAF0A3F080099000CAE4F0A374E3
:10127C0064F09000CAE0FEA3E0FFC39405EE648026
:10128C0094805009E49000CAF0A3F08014D3EF943A
:10129C005FEE6480948040099000CAE4F0A374640B
:1012AC00F07FF712BE028F3FE4F53C7B017A0079A8
:1012BC0088AD3C12C10C50121B7A00793FAD3C1228
:1012CC00C10C92617A00792480747474253CF58287
:1012DC00E43400F583E0FFB40103304D27EFB40292
:1012EC000A90000BE07002A3E060197474253CF5C1
:1012FC0082E43400F583E0B4031490000DE0700236
:10130C00A3E0700A7B007A007924C2618030747487
:10131C00253CF582E43400F583E0FCB4040D303C4C
:10132C00227B007A007924D2618013ECB405147B03
:10133C00007A007924AD3C12C10C823C9261AD3C28
:10134C0012BE6E053CE53CC3940550030212B73047
:10135C004310B220B221B222900072E07004B2238A
:10136C00B22430410EA220E433F53CA22292202478
:03137C00FF9222BB
:01137F00224B
:10BC0C0030471CE4F540E54024DBFFE54090C25C86
:10BC1C0093FD12BED60540E540C3940E40E822E4E5
:10BC2C00F540E54024DDFFE434ECFE7B007A00793E
:10BC3C004112C2B6E54024DBFFAD4112BED6054031
:07BC4C00E540C3940E40DB4C
:01BC530022CE
:02B57400C168AC
:10B5B900203979206876EF540314601014606214FE
:10B5C900606524037066852080D2A022306B0775E0
:10B5D9001F03C26B802BE51FD394004024151F90D5
:10B5E9000022E0600FE52130E6055321BF801243B8
:10B5F9002140800DE52130E0055321FE80034321E0
:10B609000185218090004BE0FFB40508900147E0D7
:10B61900F580800AEFB406062067037580FFD2A182
:0DB6290022852280D2A222852380D2A32276
:03000B0002B9A88F
:10B9A800C0E0C083C082C0D075D000C00705517503
:10B9B8008A04758CF7D269C2A0C2A1C2A2C2A390A0
:10B9C800004BE0FFB40514900146E0F520A3E0F534
:10B9D80021A3E0F522A3E0F5238016EFB406122098
:10B9E800650F20670C7520FF7521FF7522FF7523F1
:10B9F800FFAF5112B5B9D007D0D0D082D083D0E0F4
:01BA0800320B
:06B57600C167C165C1665A
:08C2ED00C252E490014CF02262
:109E4600205A03029F74C25AC2A9C2A0C2A1C2A2CA
:109E5600C2A3C2B77580FF7F057E0012C251E5809E
:109E6600F4F530D2B7AF5112B5B9D2A990014CE092
:109E7600653055307003029F51C239D267A37464AE
:109E8600F090014AE530F024FC601824FC601824A8
:109E9600F8601824D0601824C06018247E70197FDA
:109EA6000480127F02800E7F06800A7F0380067F71
:109EB6000180027F0512C158E56CD39400500990C9
:109EC6000044E06003029F51204D42900080E0B4C0
:109ED6000304D260801890007FE0B40304D260804F
:109EE6000D900081E0B40304D2608002C26030604D
:109EF6001CD24D435701AD577F0912BED690002A9A
:109F06007404F0900053F0FD7F7712BED620532ED6
:109F1600900030E06028E4FD7F1212BF6ED253D26B
:109F260066900030E0787AF6900044E07010900079
:109F36002A7404F0900053F0FD7F7712BED6D23D0E
:109F4600755C00755D01E4900021F090014CE530F0
:109F5600F0B4881590014BE0FF04F0EFD3941E4057
:0E9F66000D7F0912C158D26522E490014BF024
:019F740022CA
:10BB7500C0D1CEBBA183674F3D2D9B19273D536691
:10BB8500717065554333261C1541050405050506E9
:10BB950006060707080808090A0A0B0B0D0D0F1002
:10BBA5001112151A1E232324292B2E2F2F2B28245F
:0DBBB500211D1B191715131311100F0F0E72
:10B57C004400EB000000000124000125000126001E
:06B58C00C15CC15EC15D5F
:10B1F800C262A228302001B3500302B2849000E753
:10B20800E0FEA3E0FFE4FD12BF989261A220B330F4
:10B218006101B350477B017A0079E7A220B39264B9
:10B22800E4FD12B80730610330430620610730435C
:10B23800047FE980027FEE12BE029000E2EFF090F8
:10B2480000E2E0D3940040147B017A0079E7D264ED
:10B258007D0112B807E4FD7F0A12BF6E9000E7E097
:10B26800FEA3E0FF7D0112BF984011756D013043C8
:0CB2780006302808D23022202802D230F4
:01B2840022A7
:10B28500C262A229302101B3500302B3119000E735
:10B29500E0FEA3E0FF7D0212BF989261A221B330C8
:10B2A5006101B350477B017A0079E7A221B392642B
:10B2B5007D0212B807306103304306206107304331
:10B2C500047FEA80027FEF12BE029000E3EFF09068
:10B2D50000E3E0D3940040147B017A0079E7D2645F
:10B2E5007D0312B807E4FD7F0B12BF6E9000E7E007
:10B2F500FEA3E0FF7D0312BF984011756D02304338
:0CB3050006302908D23122202902D23162
:01B311002219
:10B31200C262A22A302201B3500302B39E9000E718
:10B32200E0FEA3E0FF7D0412BF989261A222B33037
:10B332006101B350477B017A0079E7A222B392649C
:10B342007D0412B8073061033043062061073043A1
:10B35200047FEB80027FF012BE029000E4EFF090D7
:10B3620000E4E0D3940040147B017A0079E7D264D0
:10B372007D0512B807E4FD7F0C12BF6E9000E7E076
:10B38200FEA3E0FF7D0512BF984011756D033043A7
:0CB3920006302A08D23222202A02D232D1
:01B39E00228C
:10B39F00C261A22B302301B3500302B42B9000E7FC
:10B3AF00E0FEA3E0FF7D0612BF989261A223B330A7
:10B3BF006101B350477B017A0079E7A223B392640E
:10B3CF007D0612B807306103304306206107304312
:10B3DF00047FEC80027FF112BE029000E5EFF09047
:10B3EF0000E5E0D3940040147B017A0079E7D26442
:10B3FF007D0712B807E4FD7F0D12BF6E9000E7E0E6
:10B40F00FEA3E0FF7D0712BF984011756D04304316
:0CB41F0006302B08D23322202B02D2333F
:01B42B0022FE
:10B42C00C261A22C302401B3500302B4B89000E7DF
:10B43C00E0FEA3E0FF7D0812BF989261A224B33016
:10B44C006101B350477B017A0079E7A224B392647F
:10B45C007D0812B807306103304306206107304382
:10B46C00047FED80027FF212BE029000E6EFF090B6
:10B47C0000E6E0D3940040147B017A0079E7D264B3
:10B48C007D0912B807E4FD7F0E12BF6E9000E7E055
:10B49C00FEA3E0FF7D0912BF984011756D05304386
:0CB4AC0006302C08D23422202C02D234AE
:01B4B8002271
:04C30B00759FA62252
:10BBC200E4FD7908EF5403FBA2E19291139290EF06
:10BBD2007802CEC313CE13D8F9FBAF0119EF60126E
:10BBE200EB54014205E960F2ED25E0FDEBC313FBE6
:10BBF20080E8C2A9C2A0C2A1C2A2C2A38D80C2B360
:09BC0200D2B3AF5112B5B9D2A9B9
:01BC0B002216
:10BA0900788F7602087600087601087600EF13929F
:10BA190094EFA2E19295788FE6FE08E6FF12BBC289
:10BA29007F0F7E0012C25130B2107891E6FE08E60F
:10BA3900789026F618EE36F6800DC37890E679925E
:10BA490097F618E61997F67891E6C3137991F708EE
:10BA5900E61309F7E6184670BD788FE6FE08E6FF9B
:01BA690022BA
:04AD09008E338F34C2
:10AD0D00E4FB90BB8F93FF7E00900140EEF0A3EF2C
:10AD1D00F0D39534EE95334009E490013EF0A30253
:10AD2D00ADC80BEBFF3395E0FE748F2FF58274BB2E
:10AD3D003EF583E493FAFF900140E48FF012570A39
:10AD4D00900140E0FEA3E0FFD39534EE9533405ED5
:10AD5D00EF9534FFEE9533FEEAC39FFFE49EFE9020
:10AD6D00013EF0A3EFF07C007D0A12566D90013E7E
:10AD7D00EEF0A3EFF0EAFD1256D490013EEEF0A3F3
:10AD8D00EFF07C007D0512566D7D0A1256D49001B0
:10AD9D003EEEF0A3EFF0EBFF3395E0FE7C007D057A
:10ADAD0012566D90013EEE8FF012570A800EEB6039
:10ADBD000302AD2F90013EF0A374FFF090013EE031
:04ADCD00FEA3E0FF02
:01ADD100225F
:10967A00E54125E0240BF582E43400F583E0FEA3FE
:02968A00E0FFFF
:04968C008E428F4338
:109690007B0EEB30480E3395E0FE7480240EF5828D
:1096A00074BB800CFF3395E0FE74752FF58274BB9C
:1096B0003EF583E493FF900142E4F0A3EFF0D390F2
:1096C0000143E09543900142E095424005EBFF02E3
:1096D00097C91BEBFF3395E0FE30480974802FF5E6
:1096E0008274BB800774752FF58274BB3EF583E4EA
:1096F00093FF900142E48FF012570A900142E0FE7E
:10970000A3E0FFD39543EE954250030297C0EF9537
:1097100043FFEE9542FE7C007D6412566D90014041
:10972000EEF0A3EFF0900140E0FEA3E0FFEBFD338D
:1097300095E0FC30480974802DF58274BB80077475
:10974000752DF58274BB3CF583E493FD7C001256C5
:10975000D4900140EEF0A3EFF0C3EB64809484EB6F
:10976000FF40253395E0FEEF24FCFFEE34FFFE7C46
:10977000007D6412566D900140EE8FF012570A90F2
:109780000140E0547FF080543395E0FE7C007D641E
:1097900012566D900140EE8FF012570A900140E092
:1097A000FEA3E0FFC374909FFF74019EFE900140F2
:1097B000F0A3EFF0EE4480900140F0A3EFF0801CA6
:1097C000EB60030296D2AF03EF3395E0FE7C007DA1
:1097D0006412566D900140EEF0A3EFF0900140E06E
:0497E000FEA3E0FF05
:0197E4002262
:1086D700E54175F016A4241BFFE435F0FEE54125BE
:1086E700E0240BF582E43400F583E0FCA3E0FD749D
:0F86F700E92541F582E43400F583E024FF926128
:088706008E428F438C448D4527
:10870E0075480AE54825E02F04FF12BE02EF7F00F0
:10871E00FEC006C007E54825E02543FF12BE02EF66
:10872E00FDD0E02DF54AD0E03400F549C3E545947F
:10873E00FFE544648094834009854946854A470293
:10874E008921AE44AF457C007D0A12566D7C037DB7
:10875E00FF1256D48F48E548206103028835042560
:10876E00E0254304FF12BE02EF7F00FEC006C007E5
:10877E00E5480425E02543FF12BE02EFFDD0E02DB3
:10878E00F54AD0E03400F549E54825E0254304FFDD
:10879E0012BE02EF7F00FEC006C007E54825E025A9
:1087AE0043FF12BE02EFFDD0E02DFFD0E03400FEFD
:1087BE00C3E54A9FF54AE5499EF549AF48EF339523
:1087CE00E0FE7C037DFF12566DAA06AB07AE44AFEA
:1087DE00457C007D0A12566DC3EF9BFDEE9AFC128E
:1087EE0054927B007AC0797F78441253F0C004C053
:1087FE0005C006C007AC49AD4AEC125492D003D066
:10880E0002D001D0001252E71254CB8E468F47E5AC
:10881E004825E0254304FF12BE02EF7F00FEC0068E
:10882E00C007E54802890425E0254304FF12BE0275
:10883E00EF7F00FEC006C007E54825E02543FF1286
:10884E00BE02EFFDD0E02DF54AD0E03400F549E54B
:10885E00480425E0254304FF12BE02EF7F00FEC050
:10886E0006C007E5480425E02543FF12BE02EFFDD2
:10887E00D0E02DFFD0E03400FEC3E54A9FF54AE577
:10888E00499EF549AF48EF3395E0FEEF2401FFE432
:10889E003EFE7C037DFF12566DAA06AB07AE44AFBB
:1088AE00457C007D0A12566DC3EB9FFDEA9EFC12BD
:1088BE0054927B007AC0797F78441253F0C004C082
:1088CE0005C006C007AC49AD4AEC125492D003D095
:1088DE0002D001D0001252E71254CB8E468F47E5DC
:1088EE00480425E0254304FF12BE02EF7F00FEC0C0
:1088FE0006C007E5480425E02543FF12BE02EFFD42
:10890E00D0E02DFFD0E03400FEEF2547F547EE35E1
:07891E0046F546AE46AF47E7
:01892500222F
:107EFD0090007CE0F543E4F542742D2542F582E4D3
:107F0D003400F583E064016003027F98747F25429D
:107F1D00F582E43400F583E0640160030280E33010
:107F2D005D030280E3AF43EF3395E0FE7C007D0AF5
:107F3D0012566DE54225E0240BF582E43400F583FD
:107F4D00E0FCA3E0C39FEE6480F8EC6480985005DC
:107F5D00205E02807CAF43EF3395E0FE7C007D0A0E
:107F6D0012566DE54225E0240BF582E43400F583CD
:107F7D00E0FCA3E0C39FEE6480F8EC6480984003BE
:107F8D000280E3205E030280E38070742D2542F5AC
:107F9D0082E43400F583E0FF64036008EF6405605C
:107FAD00030280E3747F2542F582E43400F583E01B
:107FBD006401704E305D030280E3E54225E0240B41
:107FCD00F582E43400F583E0FEA3E04E7010205EF0
:107FDD000D90007DE0FD7F1412BF6E0280E3E5423F
:107FED0025E0240BF582E43400F583E0FEA3E04E9A
:107FFD0060030280E3205E030280E3C25ED25D0275
:10800D0080E3747F2542F582E43400F583E0640259
:10801D0060030280E3900030E0D3940050030280AF
:10802D00E374FB2542F582E43400F583E0FFE5427D
:10803D0025E0240BF582E43400F583E0FCA3E06F2A
:10804D007001EC70030280D674D72542F582E434BA
:10805D0000F583E004F074D72542F582E43400F591
:10806D0083E0D39400406F74D72542F582E4340049
:10807D00F583E4F0E54225E0240BF582E43400F5C8
:10808D0083A3E0FF74FB2542F582E43400F583EF12
:10809D00F0E4FD7F1212BF6ED253900030E0787A7B
:1080AD00F6900132E090002AF0900053F0FD7F77BA
:1080BD0012BED6304D0543571080035357EFAD57C1
:1080CD007F0912BED6D266800D74D72542F582E4A3
:1080DD003400F583E4F00542E542C39402500302F7
:1080ED007F06900081E064017044305D030281C71A
:1080FD007B017A0079877D0212C10C500A900089AC
:10810D00E024FF92618006D2B2A2B2926120610D8D
:10811D00205E0A90007DE0FD7F1402BF6E3061038A
:10812D000281C7205E030281C7C25ED25D2290002C
:10813D0081E0640260030281C77B017A0079877D4B
:10814D000212C10C500A900089E024FF9261800652
:10815D00D2B2A2B29261900030E0D39400405BA203
:10816D0061E433FF9000FDE06F604A9000D9E004B8
:10817D00F0E0D394004043E4F09000FDEFF0E4FD17
:10818D007F1212BF6ED253900030E0787AF69001D4
:10819D0032E090002AF0900053F0FD7F7712BED6AA
:1081AD00304D0543571080035357EFAD577F0912DC
:0A81BD00BED6D26622E49000D9F08D
:0181C7002295
:10402500753C0230481E90014EE0701812BA6A9035
:10403500014EE0C394035004C23B8008D23B90017B
:10404500197405F02048030244F112A18A400302C5
:10405500493A303B03753C03E4F541E541C3953CE2
:10406500400302427F900119E0701D90002CE06032
:1040750017742D2541F582E43400F583E06403705F
:1040850061E541C39402505AE54125E024DAF58201
:10409500E43400F583E0FEA3E0FFE54125E0240BD1
:1040A500F582E43400F583EEF0A3EFF0E54125E079
:1040B50024DAF582E43400F583E0FEA3E0FFEE3375
:1040C50095E0FDFCE47B64FAF9F8125785E5412596
:1040D500E025E024EBF582E43400F5831258210253
:1040E500427AE54125E025E024EBF582E43400F54C
:1040F50083125809E47B64FAF9F812BC99A804A95B
:1041050005AA06AB07E54125E024DAF582E434008B
:10411500F583E0FEA3E0FFEE3395E0FDFC12577753
:104125008F408E3F8D3E8C3DE47F28FEFDFCAB40ED
:10413500AA3FA93EA83DC31257E2500E74FF7FD88F
:10414500FEFDFCA83D1257E2503DE54125E025E086
:1041550024EBF582E43400F583C083C08212581540
:10416500C000C001C002C003E47F0AFEFDFCAB40F5
:10417500AA3FA93EA83D125785D003D002D001D051
:104185000012576A02424690002CE024FFFFE434F7
:10419500FFFEE4FCFDE54125E025E024EBF582E4A6
:1041A5003400F583125815125785E54125E025E0C1
:1041B50024EBF582E43400F583125821E54125E02E
:1041C50025E024EBF582E43400F583C083C0821238
:1041D5005815C000C001C002C003E54125E024DA3E
:1041E500F582E43400F583E0FEA3E0FFEE3395E0CD
:1041F500FDFCE47B64FAF9F8125785D003D002D0B0
:1042050001D00012576AD082D083125821E541258A
:10421500E025E024EBF582E43400F583C083C08219
:10422500125809C004C005C006C00790002CE0FF65
:10423500E4F8F9FAAB07D007D006D005D00412BCD4
:1042450099D082D083125821E54125E025E024EB61
:10425500F582E43400F583125809E47B64FAF9F831
:1042650012BC99E54125E0240BF582E43400F58381
:10427500EEF0A3EFF00541024060303B7890000F6F
:1042850012968790013EEEF0A3EFF0EE90013E30DE
:10429500E712E0547FFEA3E0FFC3E49FFFE49E9096
:1042A500000F8008E0FFA3E090000FCFF0A3EFF030
:1042B50090003BE0602290000FE0FEA3E0FF7C0051
:1042C5007D0912566D7D051256D4EF2440FFEE345C
:1042D5000190000FF0A3EFF0900122E0FEA3E0FFB4
:1042E500900010E02FFF90000FE03ECF240CCF345C
:1042F500FEF0A3EFF0E4F541742D2541F582E43499
:1043050000F583E0FA6401707A12967A90013EEE28
:10431500F0A3EFF0EE90013E30E710E0547FFEA3EE
:10432500E0FFC3E49FFFE49EFE8005E0FEA3E0FFFF
:10433500E54125E0240BF582E43400F583EEF0A396
:10434500EFF090003BE06038E54125E0240BF58275
:10435500E43400F583E0FEA3E0FF7C007D091256FE
:104365006D7D051256D4EF2440FFEE3401FEE54184
:1043750025E0240BF582E43400F583EEF0A3EFF09D
:104385000244A2EA64027031E54125E0240BF5827E
:10439500E43400F583E0FCA3E0FDEC1254927B00CD
:1043A5007AC0797F78441253F0E4FBFA79C87842F1
:1043B5001252E71254CB0244D0742D2541F582E404
:1043C5003400F583E0FF64036008EF6405600302D1
:1043D5004475E54125E0240BF582E43400F583E0DE
:1043E500FCA3E0FDEC1254927B007AC0797F7844FF
:1043F5001253F0E4FBFA794878421252E71254CB93
:1044050090013EEEF0A3EFF0D39418EE6480948013
:10441500501D742D2541F582E43400F583E0FFB489
:104425000504D25C8034EF6403702FC25C802BC31B
:1044350090013FE0941A90013EE064809480401A18
:10444500742D2541F582E43400F583E0FFB40504BD
:10445500C25C8006EFB40302D25CA25CE433FFE5E4
:104465004125E0240BF582E43400F583E40244DEC3
:10447500742D2541F582E43400F583E06404705D14
:104485001286D790013EEEF0A3EFF0E54125E0243A
:104495000BF582E43400F583EEF0A3EFF0E541255A
:1044A500E0241EF582E43401F583E0FEA3E0FFE598
:1044B5004125E0240BF582E43400F583E0FCA3E01C
:1044C5002FFFEC3ECF240CCF34FEFEE54125E02442
:1044D5000BF582E43400F583EEF0A3EFF00541E53A
:1044E50041C3940250030242FD02493AB25B305B7C
:1044F500207F0312BA0990013EEEF0A3EFF0E0250C
:10450500E0FF90013EE033FEF0A3EFF09000DC8089
:104515001E7F0212BA0990013EEEF0A3EFF0E025EE
:10452500E0FF90013EE033FEF0A3EFF09000DAEEFD
:10453500F0A3EFF0E4F541900119E0700690002C2E
:10454500E0705AE54125E024DAF582E43400F5838C
:10455500E0FEA3E0FFE54125E0240BF582E434000D
:10456500F583EEF0A3EFF0E54125E024DAF582E4EA
:104575003400F583E0FEA3E0FFEE3395E0FDFCE4B7
:104585007B64FAF9F8125785E54125E025E024EB2F
:10459500F582E43400F583125821024735E54125BB
:1045A500E025E024EBF582E43400F583125809E4B4
:1045B5007B64FAF9F812BC99A804A905AA06AB0709
:1045C500E54125E024DAF582E43400F583E0FEA335
:1045D500E0FFEE3395E0FDFC1257778F408E3F8D5F
:1045E5003E8C3DE47F28FEFDFCAB40AA3FA93EA8DA
:1045F5003DC31257E2500E74FF7FD8FEFDFCA83D67
:104605001257E2503DE54125E025E024EBF582E433
:104615003400F583C083C082125815C000C001C0A4
:1046250002C003E47F0AFEFDFCAB40AA3FA93EA8F9
:104635003D125785D003D002D001D00012576A022F
:10464500470190002CE024FFFFE434FFFEE4FCFD6D
:10465500E54125E025E024EBF582E43400F58312FD
:104665005815125785E54125E025E024EBF582E450
:104675003400F583125821E54125E025E024EBF5CA
:1046850082E43400F583C083C082125815C000C08F
:1046950001C002C003E54125E024DAF582E43400D7
:1046A500F583E0FEA3E0FFEE3395E0FDFCE47B64DB
:1046B500FAF9F8125785D003D002D001D00012576D
:1046C5006AD082D083125821E54125E025E024EB0C
:1046D500F582E43400F583C083C082125809C00412
:1046E500C005C006C00790002CE0FFE4F8F9FAAB5E
:1046F50007D007D006D005D00412BC99D082D0834C
:10470500125821E54125E025E024EBF582E434004B
:10471500F583125809E47B64FAF9F812BC99E5416E
:1047250025E0240BF582E43400F583EEF0A3EFF0E9
:104735000541E5416402600302453CE4F541742D01
:104745002541F582E43400F583E0FA640160030253
:1047550047D412967A90013EEEF0A3EFF0EE900169
:104765003E30E710E0547FFEA3E0FFC3E49FFFE483
:104775009EFE8005E0FEA3E0FFE54125E0240BF564
:1047850082E43400F583EEF0A3EFF090003BE07097
:10479500030248EEE54125E0240BF582E43400F5FB
:1047A50083E0FEA3E0FF7C007D0912566D7D0512B6
:1047B50056D4EF2440FFEE3401FEE54125E0240BFD
:1047C500F582E43400F583EEF0A3EFF00248EEEA5B
:1047D50064027031E54125E0240BF582E43400F5EF
:1047E50083E0FCA3E0FDEC1254927B007AC079FFD4
:1047F50078441253F0E4FBFA79C878421252E71272
:1048050054CB02491C742D2541F582E43400F5830F
:10481500E0FF64036008EF640560030248C1E541F9
:1048250025E0240BF582E43400F583E0FCA3E0FDEC
:10483500EC1254927B007AC079FF78441253F0E46D
:10484500FBFA794878421252E71254CB90013EEEBA
:10485500F0A3EFF0D39418EE64809480501D742D6E
:104865002541F582E43400F583E0FFB40504D25C0C
:104875008034EF6403702FC25C802BC390013FE04E
:10488500941A90013EE064809480401A742D25416D
:10489500F582E43400F583E0FFB40504C25C8006CC
:1048A500EFB40302D25CA25CE433FFE54125E024CA
:1048B5000BF582E43400F583E402492A742D254181
:1048C500F582E43400F583E06404705D1286D790C8
:1048D500013EEEF0A3EFF0E54125E0240BF582E47F
:1048E5003400F583EEF0A3EFF0E54125E0241EF555
:1048F50082E43401F583E0FEA3E0FFE54125E024F1
:104905000BF582E43400F583E0FCA3E02FFFEC3ED9
:10491500CF240CCF34FEFEE54125E0240BF582E4DF
:104925003400F583EEF0A3EFF00541E541C39402B1
:104935005003024743E4F5417B017A007987AD4195
:1049450012C10C503FE54125E0FFC374FF9FFF12E4
:10495500BE02EF7F00FEC006C007E54125E0FFC3AC
:1049650074FE9FFF12BE02EFFDD0E02DFFD0E034B4
:1049750000FEE54125E0240BF582E43400F583EEE5
:10498500F0A3EFF00541E541C3940240AB027EFD83
:10499500E4FD7F0512BF6E789906E6D394014002C7
:1049A500E4F62041033048097899E6B40103124042
:1049B50025E5586003024BCA30415390006DE02550
:1049C500E0248BF8E6FE08E6FFC3944AEE64809483
:1049D5008150057524018013D3EF9494EE6480947F
:1049E5008240057524028003752404A22830200125
:1049F500B34002807EA229302101B34003024A85DB
:104A0500A22A302201B35003024AAF024A92900013
:104A15006DE025E0248BF8E6FE08E6FFC394C8EEBA
:104A25006480948050057524018033C3EF9490EE23
:104A35006480948150057524028023C3EF9458EE59
:104A45006480948250057524048013C3EF9420EE8E
:104A550064809483500575240880037524103043C1
:104A65000AB220B221B222B223B224A228302001F8
:104A7500B34005756D018032A229302101B340058F
:104A8500756D028025A22A302201B34005756D039C
:104A95008018A22B302301B34005756D04800BA24D
:104AA5002C302401B34003756D05900027E0700399
:104AB50002522A7899E67060900031E0FFE4FCFD2F
:104AC500FEC006C00790006DE025E0248BF8E6FEE9
:104AD50008E6FFEE3395E08F4D8E4CF54BF54AD049
:104AE50007D00612C06AE47B64FAF9F812BC999003
:104AF5000013EEF0A3EFF0D394FFEE6480948340AF
:104B05000A9000137403F0A374FFF0C3900013E040
:104B150064809480506B80657899E664017062903A
:104B25000031E0FFE4FCFDFEC006C00790006EE02A
:104B350025E02487F8E6FE08E6FFEE3395E08F4D85
:104B45008E4CF54BF54AD007D00612C06AE47B645B
:104B5500FAF9F812BC99900015EEF0A3EFF0D39492
:104B6500FFEE64809483400A9000157403F0A374EB
:104B7500FFF0C3900015E0648094805004E4F0A336
:104B8500F0205603025227900031E0FFE4FCFDFEC1
:104B9500754DE8754C03F54BF54A12C06AE47B6424
:104BA500FAF9F812BC99900013EEF0A3EFF0D39444
:104BB500FFEE64809483400A9000137403F0A3749D
:104BC500FFF002522712B1F812B28512B312204833
:104BD5000620411E20481B12B39F12B42C9000D60C
:104BE500E0FF64016004EFB40308A22B9294A22CA9
:104BF50092957899E6FF6003024DF0900046E060DB
:104C050003024FE7900027E07003024FE7204103BE
:104C1500024CB7302315EF25E02413F582E4340068
:104C2500F5837403F0A374E8F080127899E625E023
:104C35002413F582E43400F583E4F0A3F0900077C3
:104C4500E0FFB40106204D03024D22EFB4020D90A2
:104C5500000BE07002A3E07003024D22900077E0A4
:104C6500B4030D90000DE07002A3E07003024D2225
:104C7500900077E0FFB40406303C03024D32EF6448
:104C8500056003024D84303C05FE7F0180047E00F3
:104C95007F007899E6FD25E02413F582E43400F5DC
:104CA50083EEF0A3EFF04E7003024D74024D5F02E8
:104CB5004D7490006DE024FEF582E43400F583E048
:104CC50024DBFF12BE02EF5403FF7899E6BF0314FD
:104CD50025E02413F582E43400F5837403F0A3740E
:104CE500E8F0800F25E02413F582E43400F583E431
:104CF500F0A3F0900079E0FFB40103304D1FEFB44D
:104D0500020A90000BE07002A3E06011900079E0C8
:104D1500B4030F90000DE07002A3E070057899E6EA
:104D2500804E900079E0FFB40408303C057899E6A0
:104D35008029EF64057048303C05FE7F0180047EC4
:104D4500007F007899E6FD25E02413F582E4340020
:104D5500F583EEF0A3EFF04E6015ED25E02413F595
:104D650082E43400F5837403F0A374E8F08010ED59
:104D750025E02413F582E43400F583E4F0A3F02064
:104D85005603024FE4900031E0FFE4FCFDFE754D53
:104D9500E8754C03F54BF54A12C06AE47B64FAF9F1
:104DA500F812BC997899E6FD25E02413F582E434E0
:104DB50000F583EEF0A3EFF0ED25E02413F582E492
:104DC5003400F583E0FEA3E0D394FFEE6480948382
:104DD5005003024FE4ED25E02413F582E43400F599
:104DE500837403F0A374FFF0024FE47899E6FF643F
:104DF500016003024FE7900046E06003024FE79031
:104E05000027E07003024FE7204103024EB2302431
:104E150015EF25E02413F582E43400F5837403F0DF
:104E2500A374E8F080127899E625E02413F582E46E
:104E35003400F583E4F0A3F0900078E0FFB40106B8
:104E4500204D03024F1FEFB4020D90000BE07002DE
:104E5500A3E07003024F1F900078E0B4030D9000AB
:104E65000DE07002A3E07003024F1F900078E0FF91
:104E7500B40406303C03024F2FEF64056003024F74
:104E850081303C05FE7F0180047E007F007899E635
:104E9500FD25E02413F582E43400F583EEF0A3EF5D
:104EA500F04E7003024F71024F5C024F7190006D1E
:104EB500E024FEF582E43400F583E024DBFF12BE36
:104EC50002EF13135403FF7899E6BF031425E0247A
:104ED50013F582E43400F5837403F0A374E8F080DD
:104EE5000F25E02413F582E43400F583E4F0A3F004
:104EF50090007AE0FFB40103304D1FEFB4020A9031
:104F0500000BE07002A3E0601190007AE0B4030F9B
:104F150090000DE07002A3E070057899E6804E9050
:104F2500007AE0FFB40408303C057899E68029EF63
:104F350064057048303C05FE7F0180047E007F00DB
:104F45007899E6FD25E02413F582E43400F583EE37
:104F5500F0A3EFF04E6015ED25E02413F582E4345F
:104F650000F5837403F0A374E8F08010ED25E024C8
:104F750013F582E43400F583E4F0A3F03056609035
:104F85000031E0FFE4FCFDFE754DE8754C03F54B83
:104F9500F54A12C06AE47B64FAF9F812BC9978996B
:104FA500E6FD25E02413F582E43400F583EEF0A355
:104FB500EFF0ED25E02413F582E43400F583E0FEFF
:104FC500A3E0D394FFEE648094834013ED25E024A1
:104FD50013F582E43400F5837403F0A374FFF01233
:104FE500B8DC900027E0700302522A900046E0707A
:104FF5000302522A7899E660030250F0900031E0EE
:10500500FFE4FCFDFEC006C00790006DE025E0242E
:105015008BF8E6FE08E6FFEE3395E08F4D8E4CF5F6
:105025004BF54AD007D00612C06AE47B64FAF9F85A
:1050350012BC99900013EEF0A3EFF0D394FFEE6449
:10504500809483400A9000137403F0A374FFF0C3A7
:10505500900013E0648094805004E4F0A3F0900085
:1050650079E0FFB40103304D1FEFB4020A90000B45
:10507500E07002A3E06011900079E0B403109000A5
:105085000DE07002A3E07006E4900013805A9000D2
:1050950079E0FFB40408303C057899E68029EF648F
:1050A500057048303C05FE7F0180047E007F007856
:1050B50099E6FD25E02413F582E43400F583EEF04E
:1050C500A3EFF04E6015ED25E02413F582E43400DE
:1050D500F5837403F0A374FFF08010ED25E024132D
:1050E500F582E43400F583E4F0A3F07899E66401F1
:1050F50060030251E9900031E0FFE4FCFDFEC006CB
:10510500C00790006EE025E02487F8E6FE08E6FF7C
:10511500EE3395E08F4D8E4CF54BF54AD007D00612
:1051250012C06AE47B64FAF9F812BC99900015EE96
:10513500F0A3EFF0D394FFEE64809483400A9000CF
:10514500157403F0A374FFF0C3900015E064809418
:10515500805004E4F0A3F090007AE0FFB40103303E
:105165004D1FEFB4020A90000BE07002A3E060113E
:1051750090007AE0B4031090000DE07002A3E07097
:1051850006E4900015805A90007AE0FFB4040830D8
:105195003C057899E68029EF64057048303C05FEAA
:1051A5007F0180047E007F007899E6FD25E02413C9
:1051B500F582E43400F583EEF0A3EFF04E6015EDD3
:1051C50025E02413F582E43400F5837403F0A37419
:1051D500FFF08010ED25E02413F582E43400F5831B
:1051E500E4F0A3F030563B900031E0FFE4FCFDFE17
:1051F500754DE8754C03F54BF54A12C06AE47B64BE
:10520500FAF9F812BC99900013EEF0A3EFF0D394DD
:10521500FFEE64809483400A9000137403F0A37436
:10522500FFF012B8DC305F030252CFE56D70030268
:1052350052CF9000D6E0FF64046004EFB40C1290E6
:105245000072E06401600A539BEFE4FD7F1312BF17
:105255006EE56D6401600330300DA220B39228A283
:105265002892A7C2308056E56D6402600330310D87
:10527500A221B39229A22992A6C2318040E56D648C
:1052850003600330320DA222B3922AA22A9293C25E
:1052950032802AE56D6404600330330DA223B39296
:1052A5002BA22B9290C2338014E56D640560033008
:1052B500340BA224B3922CA22C9291C234E4F56D46
:1052C5007FDC7E0512C25112C30B9000D6E0FF644D
:1052D500016004EFB40308A22B9294A22C9295C20C
:0252E5005F2246
:10B8DC007899E625E02413F582E43400F583E0FE44
:03B8EC00A3E0FFD7
:10B8EF008E318F32900027E0F9B402157899E66017
:10B8FF000612AD098FAC22AF32AE3112AD098FA750
:10B90F0022E9B403157899E6AF32AE31600612AD75
:10B91F00098FA62212AD098FA522D294D295AF32EC
:10B92F00AE3112BBC27F197E0012C2517899E61355
:05B93F009294C2952264
:10B94400E4F531F532304802C322D294D295E4FFB3
:10B95400FE12BBC27F197E0012C251C294C2957FEF
:10B96400E87E0312C25112C30B0532E532AE3170C8
:10B9740002053114C394D0EE94075023E5326401D8
:10B9840045317016D294D2957FFF7E0312BBC27FDD
:10B99400327E0012C251C294C29520B2CCD322127C
:03B9A400C30BC30F
:01B9A700227D
:0300130002A64AF8
:10A64A00C0E0C0F0C083C082C0D075D000C000C0D6
:10A65A0001C002C003C004C005C006C007D25FE53E
:10A66A006D700302A71A9000D6E0FF64046004EF3D
:10A67A00B40C1B900072E064016013539BEF7FE9F6
:10A68A007E0212C251E4FD7F1312BF6E80077FE97A
:10A69A007E0212C251E56D6401600330300DA220C2
:10A6AA00B39228A22892A7C2308056E56D64026050
:10A6BA000330310DA221B39229A22992A6C2318078
:10A6CA0040E56D6403600330320DA222B3922AA2E0
:10A6DA002A9293C232802AE56D6404600330330DF6
:10A6EA00A223B3922BA22B9290C2338014E56D64FD
:10A6FA0005600330340BA224B3922CA22C9291C28F
:10A70A0034D2917FDC7E0512C25112C30B756D00E3
:10A71A00D007D006D005D004D003D002D001D00093
:0BA72A00D0D0D082D083D0F0D0E0323D
:10B5920002853232C16D048B000000000487000076
:02B5A2000000A7
:1032EC00E4FD7F0312BF6E206D0302353BE478953D
:1032FC00F67895E6FFC39406500F74262FF582E4FA
:10330C003401F583E4F00680E8E47895F67895E6E8
:10331C00FFC39406500F742C2FF582E43401F5830F
:10332C00E4F00680E8900057E0FF900056E0FE2F96
:10333C007895F6EED394004039E408F6900056E008
:10334C00FF7896E6C39F502AE6FBC3EF9B75F064AB
:10335C00A4FFAEF018E6FD7C0012567FC374649F88
:10336C00FF74262BF582E43401F583EFF078960692
:10337C0080CA900057E0D39400403AE47897F690D6
:10338C000057E0FF7897E6C39F502AE6FBC3EF9BFC
:10339C0075F064A4FFAEF07895E6FD7C0012567FC4
:1033AC00900056E02B2426F582E43401F583EFF0EF
:1033BC0078970680CA900055E0FF900054E0FE2FED
:1033CC007895F6EED394004039E408F6900054E07A
:1033DC00FF7896E6C39F502AE6FBC3EF9B75F0641B
:1033EC00A4FFAEF018E6FD7C0012567FC374649FF8
:1033FC00FF742C2BF582E43401F583EFF0789606FC
:10340C0080CA900055E0D39400403AE47897F69047
:10341C000055E0FF7897E6C39F502AE6FBC3EF9B6D
:10342C0075F064A4FFAEF07895E6FD7C0012567F33
:10343C00900054E02B242CF582E43401F583EFF05A
:10344C0078970680CAE47898F67898E6F9C39402DF
:10345C004003023539E6FB25E025E0245EF81258DE
:10346C002D00000000EB25E0FFE433FEC3742C9F1D
:10347C00FDE49EFC742B2DF58274003CF583E0FD7D
:10348C00C3742B9FFFE49EFE742B2FF58274003EB9
:10349C00F583E02D7895F6742B2FF58274003EF5AC
:1034AC0083E07008747F29F87664807BE925E0FF5F
:1034BC00E433FEC3742C9FFFE49EFE742B2FF58225
:1034CC0074003EF583E078987008E6247FF8E4F603
:1034DC008055E6FD25E0FFE433FEC3742B9FFFE42B
:1034EC009EFE742B2FF58274003EF583E0FFED7584
:1034FC00F006A42426F582E43401F583E5822FF549
:10350C0082E43583F583E0FFE6FD75F006A42426FE
:10351C00F582E43401F583E02FFFE433C313EF139A
:10352C00FF747F2DF8A607789806023455C26D7883
:10353C0077E6FE08E6FF787226FDEE1836FC7891E9
:10354C00F608EDF6C3EF787096FFEE18967893F6C2
:10355C0008A607D3E5569DEC6480F8E55564809881
:10356C004003023664C3E55678949618E66480F8F6
:10357C00E5556480985003023664E47F107E27FD85
:10358C00FCAB61AA60A95FA85ED31257E240097533
:10359C003EFF753FEC023693E4FFFEFDFCAB61AAE7
:1035AC0060A95FA85ED31257E240417877E6FE0827
:1035BC00E6FF24FFFDEE34FFFCC3E5569DEC648072
:1035CC00F8E5556480985003C380537877E6FE087D
:1035DC00E6FF2401FDE43EFCD3E5569DEC6480F847
:1035EC00E5556480985003023693805C7FF07ED85A
:1035FC007DFF7CFFAB61AA60A95FA85ED31257E286
:10360C00404E7877E6FE08E6FF2401FDE43EFCD34D
:10361C00E5569DEC6480F8E555648098400CE556C1
:10362C009FF53FE5559EF53E805D7877E6FE08E612
:10363C00FF24FFFDEE34FFFCC3E5569DEC6480F8DF
:10364C00E5556480985040C3EF9556F53FEE8033B6
:10365C00753E00753F14802FD3E55678929618E688
:10366C006480F8E555648098400FE556787896F5B7
:10367C003FE5551896F53E800EC37878E69556F5DD
:10368C003F18E69555F53ED3E53F9432E53E648010
:10369C0094804006753E00753F32900036E0FFD3B3
:1036AC00940050030237BDD3E55678929618E66421
:1036BC0080F8E555648098502BC3E556789496189D
:1036CC00E66480F8E55564809840197E00AC3EAD08
:1036DC003F12566D7C007D061256D4EE3395E0FDFC
:1036EC00FC023789D3E55678929618E66480F8E5A3
:1036FC00556480984049AE3EAF3FEE3395E0FDFCFB
:10370C00C007900036E0FFE48F4DF54CF54BF54AC1
:10371C00D00712C06AE4754D06F54CF54BF54A120C
:10372C00C292A804A905AA06C3E5619FF561E560EC
:10373C009AF560E55F99F55FE55E98F55E8052C39A
:10374C00E55678949618E66480F8E55564809850B0
:10375C0040AE3EAF3FEE3395E0FDFCC00790003627
:10376C00E0FFE48F4DF54CF54BF54AD00712C06ADB
:10377C00E4754D06F54CF54BF54A12C292E5612FF6
:10378C00F561E5603EF560E55F3DF55FE55E3CF5B6
:10379C005EE4754DE8754C03F54BF54AAF61AE60D0
:1037AC00AD5FAC5E12C2928F458E448D438C4280CD
:1037BC0009E4F545F544F543F5427891E6FE08E653
:1037CC00FFD3E5569FEE6480F8E55564809850155C
:1037DC00C3E55678949618E66480F8E555648098AD
:1037EC00400302391E900035E0D39400407BD3E5B2
:1037FC00569FEE6480F8E555648098AE3EAF3FEE80
:10380C0040343395E0FDFCE4754D64F54CF54BF517
:10381C004A12C06AC007900035E0FFE48F4DF54CAA
:10382C00F54BF54AD00712C292787FE6C39FF5415B
:10383C00E49EF540803B3395E0FDFCE4754D64F56A
:10384C004CF54BF54A12C06AC007900035E0FFE416
:10385C008F4DF54CF54BF54AD00712C292787FE6A6
:10386C002FF541E43EF5408008787FE6754000F581
:10387C0041D3E5419464E5406480948040067540F2
:10388C0000754164C3E540648094805005E4F540C4
:10389C00F541AE40EE3395E0FDFCE5412545FFEEEC
:1038AC003544FEED3543FDEC3542FCE47B64FAF91E
:1038BC00F8C31257E25005C37464801BAE40EE335C
:1038CC0095E0FDFCE5412545EE3544ED3543FDEC39
:1038DC00354233502EC3E49541FFE49540FE3395B9
:1038EC00E08F458E44F543F542E47FE87E03FDFC12
:1038FC00AB45AA44A943A8421257858F618E608DAF
:10390C005F8C5EE5412545F53DE5403544F53C02CF
:10391C0039EF7893E6FE08E6FF7891E6FC08E6FDC1
:10392C006F7002EC6E70030239DBED2FFFEC3EFE84
:10393C007C007D021256D4788FEEF608EFF6C3E5C4
:10394C00569FEE6480F8E555648098503C787FE68D
:10395C00FF900126E0C39FFDE49400FC788FE6FA0B
:10396C0008E6FBC39556FFEA9555FE12566DC3EB60
:10397C00789496FDEA1896FC1256D4787FE67C0073
:10398C002FF53DEC3EF53C804E900056E02426F59C
:10399C0082E43401F583E0FF787FE6C39FFDE49475
:1039AC0000FC788FE6FA08E6FBC3E5569BFFE5556D
:1039BC009AFE12566DC37892E69BFD18E69AFC129D
:1039CC0056D4787FE6C39FF53DE49EF53C8008789D
:1039DC007FE6753C00F53DE545253DF53DE5443577
:1039EC003CF53CC3E53C648094805007E4F53CF521
:1039FC003D8013D3E53D9464E53C6480948040069F
:103A0C00753C00753D647885A63D900058E0FFB488
:103A1C00011590002DE0FE64046007EE6401600265
:103A2C00802590000B8017EFB4021C90002EE0FF55
:103A3C0064046007EF64016002800C90000DE0F5F7
:103A4C003CA3E0F53D80077880E67886F622204D91
:103A5C000330530690002AE0700A900060E0FE905C
:103A6C00005F800890005EE0FE90005DE07C00242A
:103A7C00007890F6EC3E18F67F1212BE02EFFEE4D0
:103A8C00789026FFEE1836FEC006C0077F1112BED6
:103A9C0002EFFDD0E02D7892F6D0E0340018F67FDE
:103AAC001012BE02EFFEC37890E69400FF18E69E5B
:103ABC00FEC006C0077F0F12BE02EFFDC3D0E09D13
:103ACC007894F6D0E0940018F6D3E53D189618E6F5
:103ADC006480F8E53C6480984003023BDCC3E53D20
:103AEC0078949618E66480F8E53C6480985003025C
:103AFC003BDCE47F107E27FDFCAB65AA64A963A8C0
:103B0C0062D31257E24009753EFF753FFE023C0B33
:103B1C00E4FFFEFDFCAB65AA64A963A862D312574F
:103B2C00E24041788FE6FE08E6FF24FFFDEE34FF0D
:103B3C00FCC3E53D9DEC6480F8E53C648098500343
:103B4C00C38053788FE6FE08E6FF2401FDE43EFCBB
:103B5C00D3E53D9DEC6480F8E53C6480985003020D
:103B6C003C0B805C7FF07ED87DFF7CFFAB65AA644C
:103B7C00A963A862D31257E2404E788FE6FE08E69E
:103B8C00FF2401FDE43EFCD3E53D9DEC6480F8E5AB
:103B9C003C648098400CE53D9FF53FE53C9EF53E2E
:103BAC00805D788FE6FE08E6FF24FFFDEE34FFFC17
:103BBC00C3E53D9DEC6480F8E53C6480985040C3BF
:103BCC00EF953DF53FEE8033753E00753F02802F3B
:103BDC00D3E53D78929618E66480F8E53C648098CD
:103BEC00400FE53D789096F53FE53C1896F53E8004
:103BFC000EC37890E6953DF53F18E6953CF53E9062
:103C0C00005CE0FE90005BE07C002400FFEC3EFEDC
:103C1C00D3EF9400EE648094805003023D84D3E58E
:103C2C003D78929618E66480F8E53C648098503DA7
:103C3C00C3E53D78949618E66480F8E53C6480987A
:103C4C00402BAC3EAD3F12566D7C007D061256D417
:103C5C00EE3395E0FDFCE5612FF561E5603EF56026
:103C6C00E55F3DF55FE55E3CF55E023D64D3E53D09
:103C7C0078929618E66480F8E53C6480984068AECB
:103C8C003EAF3FEE3395E0FDFCC004C006C007908C
:103C9C00005CE0FE90005BE07C002400FFEC3EFE4C
:103CAC003395E08F4D8E4CF54BF54AD007D006D0AE
:103CBC000412C06AE47B0AFAF9F8125785E4754DD0
:103CCC0006F54CF54BF54A12C292A804A905AA06B2
:103CDC00C3E5659FF565E5649AF564E56399F5635D
:103CEC00E56298F5628071C3E53D78949618E664B8
:103CFC0080F8E53C648098505FAE3EAF3FEE339564
:103D0C00E0FDFCC004C006C00790005CE0FE900023
:103D1C005BE07C002400FFEC3EFE3395E08F4D8E83
:103D2C004CF54BF54AD007D006D00412C06AE47BA0
:103D3C000AFAF9F8125785E4754D06F54CF54BF572
:103D4C004A12C292E5652FF565E5643EF564E563BC
:103D5C003DF563E5623CF562E4754DE8754C03F5A1
:103D6C004BF54AAF65AE64AD63AC6212C2928F453F
:103D7C008E448D438C428009E4F545F544F543F5BA
:103D8C00427891E6FC08E6FDD3E53D9DEC6480F8B5
:103D9C00E53C6480985015C3E53D78949618E6642C
:103DAC0080F8E53C6480984003023F2690005AE07E
:103DBC00FE900059E07A002400FFEA3EFED3EF9417
:103DCC0000EE648094805003023E7ED3E53D9DEC72
:103DDC006480F8E53C648098AE3EAF3FEE404A33D9
:103DEC0095E0FDFCE4754D64F54CF54BF54A12C0BD
:103DFC006AC004C006C00790005AE0FE900059E06B
:103E0C007C002400FFEC3EFE3395E08F4D8E4CF58C
:103E1C004BF54AD007D006D00412C2927880E6C384
:103E2C009FF541E49EF54080513395E0FDFCE4752F
:103E3C004D64F54CF54BF54A12C06AC004C006C07F
:103E4C000790005AE0FE900059E07C002400FFEC43
:103E5C003EFE3395E08F4D8E4CF54BF54AD007D096
:103E6C0006D00412C2927880E62FF541E43EF5406C
:103E7C0080087880E6754000F541D3E5419464E50F
:103E8C0040648094804006754000754164C3E540F1
:103E9C00648094805005E4F540F541AE40EE3395D6
:103EAC00E0FDFCE5412545FFEE3544FEED3543FDD7
:103EBC00EC3542FCE47B64FAF9F8C31257E2500586
:103ECC00C37464801AAE40EE3395E0FDFCE54125E9
:103EDC0045EE3544ED3543EC354233502EC3E49575
:103EEC0041FFE49540FE3395E08F458E44F543F554
:103EFC0042E47FE87E03FDFCAB45AA44A943A842FB
:103F0C001257858F658E648D638C62E5412545F56E
:103F1C003DE5403544F53C023FFD7893E6FE08E66E
:103F2C00FF7891E6FC08E6FD6F7002EC6E70030200
:103F3C003FE9ED2FFFEC3EFE7C007D021256D4785B
:103F4C008FEEF608EFF6853C3E853D3FC3E53F9F7F
:103F5C00EE6480F8E53E648098503C7880E6FF90F3
:103F6C00012CE0C39FFDE49400FC788FE6FA08E690
:103F7C00FBC3953FFFEA953EFE12566DC3EB78945A
:103F8C0096FDEA1896FC1256D47880E67C002FF544
:103F9C003DEC3EF53C804E900054E0242CF582E440
:103FAC003401F583E0FF7880E6C39FFDE49400FCC8
:103FBC00788FE6FA08E6FBC3E53F9BFFE53E9AFEE9
:103FCC0012566DC37892E69BFD18E69AFC1256D4F5
:103FDC007880E6C39FF53DE49EF53C80087880E64A
:103FEC00753C00F53DE545253DF53DE544353CF595
:103FFC003CC3E53C648094805007E4F53CF53D807F
:10400C0013D3E53D9464E53C648094804006753C94
:08401C0000753D647886A63DA5
:014024002279
:1066420000C1814001C0804101C0804100C1814040
:1066520001C0804100C1814000C1814001C0804130
:1066620001C0804100C1814000C1814001C0804120
:1066720000C1814001C0804101C0804100C1814010
:1066820001C0804100C1814000C1814001C0804100
:1066920000C1814001C0804101C0804100C18140F0
:1066A20000C1814001C0804101C0804100C18140E0
:1066B20001C0804100C1814000C1814001C08041D0
:1066C20001C0804100C1814000C1814001C08041C0
:1066D20000C1814001C0804101C0804100C18140B0
:1066E20000C1814001C0804101C0804100C18140A0
:1066F20001C0804100C1814000C1814001C0804190
:1067020000C1814001C0804101C0804100C181407F
:1067120001C0804100C1814000C1814001C080416F
:1067220001C0804100C1814000C1814001C080415F
:1067320000C1814001C0804101C0804100C181404F
:1067420000C0C101C30302C2C60607C705C5C4040F
:10675200CC0C0DCD0FCFCE0E0ACACB0BC90908C87F
:10676200D81819D91BDBDA1A1EDEDF1FDD1D1CDC6F
:1067720014D4D515D71716D6D21213D311D1D010DF
:10678200F03031F133F3F23236F6F737F53534F4CF
:106792003CFCFD3DFF3F3EFEFA3A3BFB39F9F8383F
:1067A20028E8E929EB2B2AEAEE2E2FEF2DEDEC2C2F
:1067B200E42425E527E7E62622E2E323E12120E09F
:1067C200A06061A163A3A26266A6A767A56564A48F
:1067D2006CACAD6DAF6F6EAEAA6A6BAB69A9A868FF
:1067E20078B8B979BB7B7ABABE7E7FBF7DBDBC7CEF
:1067F200B47475B577B7B67672B2B373B17170B05F
:10680200509091519353529296565797559594544E
:106812009C5C5D9D5F9F9E5E5A9A9B5B99595898BE
:10682200884849894B8B8A4A4E8E8F4F8D4D4C8CAE
:10683200448485458747468682424383418180401E
:10684200000000000001000100020002000300033A
:10685200000400040005000500060006000700070A
:10686200000800080102000900AE000F000B001032
:10687200000C0011000D0012000A001300F8000ABB
:1068820000F9006500FA006600FB006700FC006882
:1068920000FE006A00FF006B0101006C004B006DFE
:1068A200004D006E004F006F0055007000590072DD
:1068B200005A0073005B0076005D0077005E00788E
:1068C200005F00790060007A0061007B0062007C5A
:1068D2000065007D0066007E0067007F0068008022
:1068E20000690081006C0083006D0084006E0085E9
:1068F20000720086007300870075008800770089A7
:1069020000B1008A00B2008B00B3008C00B4008D8D
:1069120000B5008E00B6008F00B7009000B800915D
:1069220000B9009200BA009300BB009400BC00952D
:1069320000BD009600BE009700BF009800C00099FD
:1069420000C1009A00C2009B00C3009C00C4009DCD
:1069520000C5009E00C6009F00C700A000C800A19D
:1069620000C900A200CA00A300CB00A400CC00A56D
:1069720000CD00A600CE00A700CF00A800D000A93D
:1069820000D100AA00D200AB00D300AC00DB00AD06
:1069920000DC00AE00DD00AF00DE00B000DF00B1C1
:1069A20000E000B200E100B300F300B400F400B56F
:1069B200006300B6006400B7000900B8005600B9D1
:1069C200006A00BA006B00BB005100BC005200BD5F
:1069D200005300BE00E900BF00EA00C000EB00C1A6
:1069E20000EC00C200ED00C300EE00C400EF00C5E1
:1069F20000F000C600F100C700F200C8005700C94D
:106A0200005800CA006F00CB008500CC008600CD84
:106A1200008700CE008800CF008900D0008A00D114
:106A2200008B00D2005400D3010300D4005000D5E3
:106A3200005C00D6010A00D7010B00D8004900D93A
:106A4200004700DA001B00DB001D00DC001F00DD38
:106A5200002100DE002300DF002500E0002700E126
:106A6200002900E2002B00E3002D00E4002F00E5E6
:106A7200003100E6003300E7003500E8003700E9A6
:106A8200003900EA003B00EB003D00EC003F00ED66
:106A9200004100EE004300EF004500F0007C00F1F1
:106AA200000F00F2001100F3007D00F4007F00F5FA
:106AB200008100F6008C00F7008D00F8008E00F9CE
:106AC200008F00FA009000FB009100FC009200FD94
:106AD20000D400FE00D500FF00D6010000D701015E
:106AE20000D8010200D9010300DA010400E2010525
:106AF20000E3010600E4010700E5010800E60109E0
:106B020000E7010A00E8010B0078010C0079010D91
:106B120000FD010E0013010F0015011000170111F5
:106B22000019011200830113007A0114007B011580
:106B32000100011600700117009301180094011959
:106B42000095011A0096011B0097011C010C011D02
:106B52000098011E0099011F009A0120009B01214B
:106B6200009C0122009D0123009E0124009F01251B
:106B72000104012600A0012700A1012800A2012989
:106B820000A3012A00A4012B00A5012C00A6012DBF
:106B920000A8012E00AA012F0105013001060131D2
:106BA20001070132010801330109013400AB01354B
:106BB20000AC013600AD0137010D0138010E01397B
:106BC200010F013A0110013B0111013C00AF013DEF
:106BD20000B0013E00F5FFFF00F6FFFF00F7FFFFE8
:0FB5A40041013301010B0041013BFE020800E8A9
:06ADD200FFEC3EFE7B00D9
:04ADD8008E428F43D5
:10ADDC00E4FDFC90008AE0B40117D3E5439464E5EC
:10ADEC00429400400C74BF2543F54374633542F51F
:10ADFC0042D3E543940AE5429400400BD3E54394D7
:10AE0C000EE54294004016C3E5439414E5429400C9
:10AE1C00400ED3E5439463E542940050037F002237
:10AE2C00D3E5439463E5429400400AE543249CFD3A
:10AE3C00E54234FFFCC3ED9509EC9508504BEDAEA3
:10AE4C00047802C333CE33CED8F92444F582746827
:10AE5C003EF583740193B54329E493B54224EDAEDA
:10AE6C00047802C333CE33CED8F92442F582746809
:10AE7C003EF583E493FF740193CF8FF012574B7F11
:0BAE8C0001220DBD00010C80AC7F0016
:01AE97002298
:0EC26A00C292E4F50BF5129000A2741BF022B4
:0CC29E00C292E4F50BF5127F0902C27891
:0BC2CD00C26AD2927F0A7E0002C251BA
:0300230002A8FA36
:10A8FA00C0E0C0F0C083C082C0D075D000C000C024
:10A90A0001C002C003C004C005C006C007209803E6
:10A91A0002A9B4E50BC3940C500AAF0B050B7413D0
:10A92A002FF8A699C298E50BB40105750E08802088
:10A93A00E50BB40420E515FE7C00E42516FFEC3E89
:10A94A00FEEF640A4E706AE51464067064750E0CB4
:10A95A00850C0F805CE50BB40714E5146410705184
:10A96A00E5192409F50EE5192408F50F8043E50BCE
:10A97A00B50E12E51464036018E51464066012E566
:10A98A00146410600CE50B64067026E514641970F3
:10A99A0020750F00128B6B500C751002751202D2C3
:10A9AA006BD23A800C7512018007309904C299D291
:10A9BA006AD007D006D005D004D003D002D001D087
:0CA9CA0000D0D0D082D083D0F0D0E0329A
:10C19D00E512B4020C12C2CD12C2FD121380126050
:04C1AD003202C29EFA
:108B6B00E513F4600E90013BE065136006E51360BE
:108B7B0002C322E514641970797F0412BF079001B8
:108B8B0044EEF0FCA3EFF0FDE517FE7A00E42518A8
:108B9B00FFEA3EFEEF6D7002EE6C6002C322E5153C
:108BAB00C395164004AF168002AF15E515C3951695
:108BBB004004AE158002AE1690013BE0FDC39F4012
:108BCB0005EDD39E4002C322AF517E0012BD14129D
:108BDB00BCDD7C007D0A1256D48D4FE4F54EE54E7C
:108BEB00C3954F500B7F147E0012C251054E80EE81
:108BFB00D322E5146403600EE51464066008E514E3
:108C0B0064106002C322E515FE7C00E42516FFEC20
:108C1B003EFEEF640A4E6003028CD4E514640670CA
:108C2B002890001AE065196002C32290001BE065D2
:108C3B001A6002C32290001CE0651B6002C32290E5
:108C4B00001DE0651C6002C322E514B4031912BCBD
:108C5B00DD7C007D0A1256D47E007F02CFCDCFCEB5
:108C6B00CCCE1256D48F11E5116401603690013CC5
:108C7B00E004F0E075F00584E5F07025F075110166
:108C8B0012BCDD7C007D0A1256D48D4FE4F54EE507
:108C9B004EC3954F50337F4B7E0012C251054E8011
:108CAB00EEC322E490013CF012BCDD7C007D0A1285
:108CBB0056D48D4FE4F54EE54EC3954F500B7F4B7D
:108CCB007E0012C251054E80EEE5146406705DE520
:108CDB0015FE7C00E42516FFEC3EFEC3EF9405EE7B
:108CEB009400400CEF64084E6006EF64074E703C36
:108CFB00E516C39402500990013AE030E02EC322EE
:108D0B00E516C39404500990013AE030E11EC322EA
:108D1B00E516B4080990013AE030E210C322E516DB
:108D2B00B4070990013AE030E302C322E518B4A17D
:108D3B000CE516B41007E513B4FF02C322E50E24AD
:108D4B00FEFF12BF07900144EEF0FCA3EFF0FD74A1
:108D5B0011250EF8E6FE7412250EF8E67A002400B3
:0F8D6B00FFEA3EFEEFB50506EEB50402D322C3C4
:018D7A0022D6
:0CC2AA00306AFDE4F599C26AFF02C0F2A0
:0AC2E300306AFD8F99C26A02C0F2B2
:10603200E4F53EE514B40621E4F53EE53EC3950ED3
:1060420040030266417413253EF8E6F599C26A12CE
:10605200C30B306AFD053E80E2E5146410703DF525
:106062003E7434253EF582E43401F583E0F53FF5D4
:1060720099C26A12C30B306AFDAF3F12C0F2053EED
:10608200E53EC3940640DA850A99C26A306AFD8504
:106092000D99C26A306A0302664180F8E51464030E
:1060A20060030265F085183C12C0E885143F306A2F
:1060B200FD12C0EBE53C25E0F53FE5157008E5165D
:1060C200B40A03753F06306AFD12C0EBE53EC39584
:1060D2003C40030265DBE515FE7C00E42516FFEC7F
:1060E2003EFEEF253E7A00794012ADD2EF700302F8
:1060F20065CDC3E54194F3E540648094804003029A
:1061020061F1E541944DE54064809480500DC3E512
:1061120041940FE54064809480502AC3E541947D08
:10612200E54064809480400DD3E5419483E540646A
:106132008094804010E54164A645406008E54164D2
:10614200A84540700BE54104FF12BE028F3F800359
:10615200E4F53F306AFD12C0EBE5416473454060EF
:1061620008E54164754540702AE54104FF12BE020C
:10617200EF7F00FEC006C007AF4112BE02EFFDD0A6
:10618200E02DFFD0E03400FE7C007D0A1256D48F51
:106192003F8056E54164094540702AAF4112BE0274
:1061A2008F3F533FEFE55730E305433F08800353EA
:1061B2003FF790002AE0D394004005433F01802935
:1061C200533FFE8024E54164AD454070157B017A62
:1061D2000079877D0112C10C4008900089E0F53FEB
:1061E2008007AF4112BE028F3F306AFD0265C6E5ED
:1061F200418540F01258A9636C00F363AD00F4636B
:106202002000F8626D00F9627D00FA62D200FB6341
:106212005300FC636100FD63F100FE641C00FF6437
:1062220064010064DE010164BB010264F7010364DE
:10623200CA01046500010565130106651D010765B4
:1062420027010865310109653F010A6573010B6485
:10625200AC010C65A7010D65A7010E65A7010F65CD
:10626200A7011065A70111000065CBE555F53FAF09
:106272003F12C2E3E556F53F0263EC7B017A0079F7
:10628200887D0512C10C50097FFB12BE028F3F8030
:106292001190006DE025E0248BF9E7FF3395E0EFE4
:1062A200F53F306AFD12C0EB7B017A0079887D05EB
:1062B20012C10C50097FFA12BE028F3F800C90006F
:1062C2006DE025E0248CF9E7F53F306AFD0265C6F2
:1062D2007B017A0079887D0612C10C50097FF91280
:1062E200BE028F3F800E90006EE025E02487F9E722
:1062F200FFEFF53FAF3F12C2E37B017A0079887D61
:106302000612C10C50097FF812BE028F3F800C901A
:10631200006EE025E02488F9E7F53F0263EC12C243
:10632200AAE4F53F306AFD12C0EBE5186401600390
:106332000265D690001AE0FF12C2E390001BE0FF54
:1063420012C2E390001CE0FF12C2E390001D02653E
:106352001912C2AA7885E6F53F306AFD0265C612B7
:10636200C2AA7886E6F53F0264FD7B017A0079874E
:10637200E4FD12C10C50097FFF12BE028F3F80085C
:1063820090000BE0FFEFF53FAF3F12C2E37B017AD3
:10639200007987E4FD12C10C50097FFE12BE028F04
:1063A2003F800690000CE0F53F803F7B017A007948
:1063B200877D0112C10C50097FFD12BE028F3F8002
:1063C2000890000DE0FFEFF53FAF3F12C2E37B0103
:1063D2007A0079877D0112C10C50097FFC12BE023E
:1063E2008F3F800690000EE0F53FAF3F0265391205
:1063F200C2AA787DE6FE08E6FFE4FD12BF98E43308
:10640200F53F787BE6FE08E6FFE4FD12BF985004F4
:10641200053F053F306AFD0265C612C2AA9000FE22
:10642200E0FFC39404400DEFD394065007EF240A13
:10643200F53F8028EFC39407400DEFD3940950072E
:10644200EF24FDF53F8015EFC3940A400DEFD3947E
:106452000C5007EF2407F53F80028F3F306AFD02A0
:1064620065C612C2AA9000FFE0FFC39404400DEF7C
:10647200D394065007EF240AF53F8028EFC3940710
:10648200400DEFD394095007EF24FDF53F8015EF3F
:10649200C3940A400DEFD3940C5007EF2407F53F45
:1064A20080028F3F306AFD0265C612C2AA9000CBFD
:1064B200E0F53F306AFD0265C612C2AA90014EE0C5
:1064C200F53F306AFD0265C6E55CF53F306AFD12B4
:1064D200C0EBE55DF53F306AFD0265C612C2AA3027
:1064E200430585253F8005E525F4F53F533F1F30E1
:1064F2006AFD0265C612C2AA787AE6FF803912C224
:10650200AA90014AE0FF12C2E3E490014AF0026558
:10651200D612C2AA900146E0FF801C12C2AA9001C4
:1065220047E0FF801212C2AA900148E0FF800812E1
:10653200C2AA900149E0FF12C2E30265D6D39000DD
:1065420012E094B8900011E06480948B4007740BC1
:10655200F0A374B8F0900011E0FF3395E0EFF53F3F
:10656200306AFD12C0EB900012E0F53F306AFD8008
:1065720053D3900010E094B890000FE06480948BA5
:106582004007740BF0A374B8F090000FE0FF33954E
:10659200E0EFF53F306AFD12C0EB900010E0F53FEE
:1065A200306AFD801F12C2AA7FF712BE028F3D7BA6
:1065B200007A00793DE54124F3FD12C10CE433F584
:1065C2003F306AFD12C0EB800B800012C2AAE4F5D4
:1065D2003F12C2AA053E0260CE306AFD850A99C208
:1065E2006A306AFD850D99C26A206A5380FBE51400
:1065F2006419704B12C0E885143F306AFD12C0EB7B
:1066020090013BE0F53F306AFD12C0EB90001AE0CA
:10661200FF12C2E390001BE0FF12C2E390001CE0F5
:10662200FF12C2E390001DE0FF12C2E3306AFD8553
:0F6632000A99C26A306AFD850D99C26A306AFD05
:016641002236
:1013800090003BE0F537900037E0F538E514B410F5
:1013900024E4F53574132535F8E6FF74342535F566
:1013A00082E43401F583EFF00535E535B406E585D3
:1013B0001A17851B18E51464066009E514641060AB
:1013C000030223AEE515FE7C00E425167A00793988
:1013D00012ADD2EF70030223AEC3E53A94F3E539C0
:1013E000648094804003021F81AD18AF3AAE391279
:1013F0008F784003021F6FC3E53A944FE53964804C
:101400009480401AE53A94B1E53964809480500E96
:1014100074DC253AF582E434FFF583E518F0E53A0B
:10142000640945396007AF3AAD1812BED6E53A45B2
:10143000396008E53A640245397009E53A04FFADC0
:101440001712BED6E53A640645397016E5186009EC
:10145000F4600690013BE518F07D067CEFE4FF1296
:10146000C0C8D3E53A9445E539648094805016C3EA
:10147000E53A940FE539648094804009E53A04FF29
:10148000AD1712BED6D3E53A9483E53964809480D3
:10149000500DC3E53A947DE539648094805010E5A1
:1014A0003A64A645396008E53A64A845397017AF33
:1014B0003A74DD2FF582E434FFF583E517F0EF048D
:1014C000FFAD1712BED6E53A640B4539600302152D
:1014D0007A900133E518F0647F700302157AC2AF89
:1014E000C2A9C2AAE4F59F753B76AF3B12C1221296
:1014F000C30BD2A9D2AAD2AFE518649F7041C2AF84
:10150000C2A9C2AAF59FFD7CEC7F5512C0C87D011F
:101510007CEC7FAA12C0C8E4F535AF3512BE028F4D
:1015200036E5352402FDE434ECFC12C0C80535E58F
:1015300035C3944F40E412C30BD2A9D2AAD2AF90C4
:101540000133E0FF648E6005EF648F702D90013AE7
:1015500074F3F0FD7FFF12BED6E518B48E02D24FB1
:10156000D238126032127BB87BFF7DFF7FFF12C240
:101570008B7F887E1312C25180FED3E53A9401E539
:101580003964809480500890013AE044018013D37C
:10159000E53A9403E53964809480500D90013AE077
:1015A0004402F0FD7FFF12BED6E53A64094539607A
:1015B00003021666900081E06404606890007FE09A
:1015C00064046060A3E06404605AA24DE433FFE564
:1015D0001854016F604EE51854116014D24D4357F2
:1015E0001190002A7404F0900132F012C13E801F65
:1015F00090013DE064056017C24D5357FEE4900032
:101600002AF0C253787AF6900053E0900132F0ADA0
:10161000577F0912BED690002AE0FD900053F07F5C
:101620007712BED690013DE518F0E5575404FFE56A
:101630001854046F6030E51830E20C435704AD577E
:101640007F0912BED6801F5357FBAD577F0912BECC
:10165000D61260327BFF7DFF7FFF12C28B7F887EB8
:101660001312C25180FEE53A6408453970089001B2
:101670003AE044048024E53A646E45397008AF18B6
:1016800012C038021D9FE53A640745397013900077
:10169000D6E518F090013AE04408F0FD7FFF021C07
:1016A00050E53A64604539703190002AE0FF6404E7
:1016B0007003021D9F90003CE0FEEFD39E5003029A
:1016C0001D9FE090002AF0900053E0900132F0E47A
:1016D000900053F0FD7F77021C50E53A647745395E
:1016E0007053900053E0FF90002AF012B00A90006F
:1016F0002AE070115357FEC24DAD577F0912BED676
:10170000C253E48016900030E0D394004010E4FD12
:101710007F1212BF6ED253900030E0787AF612C278
:101720003E156C9000A0740FF0E4FD7F0712BF6EB1
:101730007F01021D07E53A644F4539701E9001197B
:101740007405F090002BE0D394005003021D9F908D
:10175000002D7401F0FD7F51021C50E53A647C4578
:10176000397061900058E0B40128E4F535AF3505D3
:101770003574742FF582E43400F583E0B402041567
:10178000358007E535C3940740E3E535C394070288
:101790001D9F900058E064026003021D9FF535AF65
:1017A00035053574742FF582E43400F583E0B40315
:1017B0000415358007E535C3940740E3E535C39448
:1017C00007021D9FE53A645B4539702E900037E0B3
:1017D000653860267F0912BE02EF30E203021D9FCA
:1017E000D23E127BB81260327BFF7DFF7FFF12C2B8
:1017F0008B7F887E1312C25180FEE53A64724539B0
:10180000702DE518D3940040267F0912BE02EF30F8
:10181000E203021D9FD23E127BB81260327BFF7D35
:10182000FF7FFF12C28B7F887E1312C25180FEE5BC
:101830003A645F4539704A90003BE0653760427F0B
:101840000912BE02EF30E203021D9F7F5612BE0254
:101850008F0B7F4F12BE028F38D23E127BB8AD0B7A
:101860007F5612BED6AD387F4F12BED61260327B85
:10187000FF7DFF7FFF12C28B7F887E1312C25180D3
:10188000FEE53A64684539704AE5186402600BE584
:101890001864046005E518B40509900038E070127A
:1018A000048008900038E0B40108E4F0FD7F5C1289
:1018B000BED67F0912BE02EF30E203021D9F126006
:1018C000327BFF7DFF7FFF12C28B7F887E1312C2A7
:1018D0005180FEE53A646F45397019E518B4020A83
:1018E000E4FD7F1612BF6E021D9F7F1612C278C2E2
:1018F00068021D9FE53A645C4539704FE518640342
:101900006005E518B40211900081E0640560097477
:1019100005F0FD7FA512BED6E518B4041190002D88
:10192000E0640160097401F0FD7F5112BED6E51834
:1019300064056003021D9F90002EE06401700302A5
:101940001D9F7401F0FD7F52021C50E53A64A545CD
:10195000397067E518B40312900038E06402603F04
:10196000E06403603A7402F0802F900038E0640273
:101970006005E064037028900044E064026009E0C0
:1019800064046004E0B405089000387401F0800538
:10199000E4900038F0900038E0FD7F5C12BED6E5A0
:1019A0001864036009E51864046003021D9F900039
:1019B000437402F0FD7F67021C50E53A644B4539E1
:1019C0007010E517FE7C00E42518FFEC3E90012422
:1019D0008044E53A644D45397026E517FE7C00E405
:1019E0002518FFEC3E90011EF0A3EFF0E53A04FF4E
:1019F000AD1712BED690002DE0B40402804E8023B5
:101A0000E53A644945397021E517FE7C00E4251864
:101A1000FFEC3E900122F0A3EFF0E53A04FFAD1792
:101A200012BED61281C8021D9FE53A64474539703F
:101A300021E517FE7C00E42518FFEC3E900120F024
:101A4000A3EFF0E53A04FFAD1712BED6124025020F
:101A50001D9FE53A64A345397016E518C3940250FA
:101A600003021D9F90002D7403F0FD7F51021C5056
:101A7000E53A64A445397016E518C3940250030290
:101A80001D9F90002E7403F0FD7F52021C50E53A1A
:101A9000647345396003021C22900049E0FFE51899
:101AA000C39F5002800F900048E0FFE518D39F408D
:101AB000028002AF187E007C007D0A12566D8E31C6
:101AC0008F32E531FF3395E0EFF537E532F53890A9
:101AD000004FE538F0FD7F7312BED6900050E53719
:101AE000F0FD7F7412BED6E537FE7C00E42538F5A4
:101AF00032EC3EF531D3E53294E7E53164809483EE
:101B0000400EAE31AF327D0A1256D412AF5C800760
:101B1000AF32AE3112A28612C23E156C9000A07494
:101B20000FF0E4FD7F0712BF6E7F0112C2789000B4
:101B300044E064036003021BDA900052E0FE900070
:101B400051E07C002400FDEC3EFCE537FE7A00E429
:101B50002538FFEA3EFED3EF9DEC6480F8EE64800A
:101B6000985077E538F0FD7F7512BED6900052E5AB
:101B700037F0FD7F7612BED6900052E0FE90005105
:101B8000E07C002400FDEC3EFC900050E0FE900064
:101B90004FE07A002400FFEA3EFEEF6D7002EE6C2B
:101BA0006003021D9F900052E0FE900051E07C0017
:101BB0002400FFEC3ECF240AF532E43FF531E53254
:101BC00090004FF0FD7F7312BED6E531FF3395E0F4
:101BD000EF900050F0FD7F748076900044E0640147
:101BE0006003021D9F900050E0FE90004FE07C00DB
:101BF0002400FFEC3EFE90003AE0FDC3EF9DF5327D
:101C0000EE9CF531FF3395E0EF900052F0E5329015
:101C10000051F0FD7F7512BED6900052E0FD7F7638
:101C2000802EE53A64694539702C90002AF05357AC
:101C3000FEC24DAD577F0912BED6C253E4787AF684
:101C4000900053E0900132F0E4900053F0FD7F7774
:101C500012BED6021D9FE53AF44539700990013A4B
:101C6000E518F0021D9FE53A6456453970217F0959
:101C700012BE02EF30E203021D9F1260327BFF7D35
:101C8000FF7FFF12C28B7F887E1312C25180FEE558
:101C90003A649645397034900072E0B4011CA37424
:101CA00001F0FD7F9712BED6D2CAE4FD7F0412BFB9
:101CB0006ED24678797602021D9FE4900073F0FDA3
:101CC0007F9712BED6C2CA7F04803CE53A6497452E
:101CD00039703A900073E0B4011E9000727401F004
:101CE000FD7F9612BED6D2CAE4FD7F0412BF6E7885
:101CF000797602D246021D9FE4900072F0FD7F9635
:101D000012BED6C2CA7F0412C278021D9FE53A6491
:101D1000A645397044E517603CE5186038900085A9
:101D2000E0FE900084E07C002400FFEC3EFEE4FD39
:101D3000900007125821C23CE4900029F09000CC9A
:101D4000F0FFFEFDFC900007125815D31257F84023
:101D50004ED254804AC2548046E53A64A845397050
:101D60003EE5176038E5186034900085E0FE90008D
:101D700084E07C002400FFEC3EFEE4FD90000712AE
:101D80005821C23CE4900029F09000CCF0900083F0
:101D9000E0600C900082E06006D2548002C254D30E
:101DA000E53A9481E53964809480500DC3E53A9416
:101DB00078E539648094805013E53A640F453960C2
:101DC0000BE53A641145396003021E63D26DE53AB2
:101DD00064784539701D900055E0FF900054E02F65
:101DE000F535D39406407C74069F900054F0FD7F37
:101DF00078806DE53A64794539701D900055E0FFB3
:101E0000900054E02FF535D394064057E0FF740658
:101E10009FA3F0FD7F798048E53A647A4539701DCB
:101E2000900057E0FF900056E02FF535D394064020
:101E30003274069F900056F0FD7F7A8023E53A6465
:101E40007B4539701E900057E0FF900056E02FF55B
:101E500035D39406400DE0FF74069FA3F0FD7F7B11
:101E600012BED6E53A645945396028E53A645A45C8
:101E7000396020E53A645D45396018E53A645E45AD
:101E8000396010E53A646145396008E53A646245B5
:101E9000397005D26D021F6FE53A641B4539600841
:101EA000E53A642F4539705B7F3012BE02EF7F0048
:101EB000FEC006C0077F2F12BE02EFFDD0E02DFF4F
:101EC000D0E03400FEC006C0077F1C12BE02EF7FC8
:101ED00000FEC006C0077F1B12BE02EFFDD0E02D42
:101EE000FDD0E03400FCD007D006C3ED9FEE648047
:101EF000F8EC64809850059000E98069E49000E96E
:101F0000F0806CE53A643145396008E53A6445454E
:101F100039705C7F4612BE02EF7F00FEC006C0072C
:101F20007F4512BE02EFFDD0E02DFFD0E03400FE71
:101F3000C006C0077F3212BE02EF7F00FEC006C09F
:101F4000077F3112BE02EFFDD0E02DFDD0E034005E
:101F5000FCD007D006C3ED9FEE6480F8EC64809857
:101F600050089000EA7401F08005E49000EAF01255
:101F700040251297E51232EC12028C1289260223B8
:101F8000AEE53A8539F01258A920FF00F3217C0014
:101F9000F4232300F81FE100F922BD00FA22DB0040
:101FA000FB230000FE22F901012344010323A401C5
:101FB00004235B01062360010723650108236A01EE
:101FC0000921F9010A225B010B2372010D23720121
:101FD0000E2372010F2372011023720111000023DE
:101FE000AEE517FE7C00E42518F532EC3EF53190A5
:101FF000002BE0704EC3E5329556F534E53195552A
:10200000F533900125E02534FF900124E03533FEBF
:10201000D3EF9400EE940050030223AEEF94E8EE69
:10202000940340030223AEE5338534F012570A903F
:102030000125E0FD7F4B12BED6900124E0FD7F4CD0
:102040000220F690002BE06401705590002DE064B2
:1020500004604DC3E5329556F534E5319555F533B9
:1020600090011FE02534FF90011EE03533FED3EFD1
:102070009400EE940050030223AEEF94E8EE940334
:1020800040030223AEE5338534F012570A90011F56
:10209000E0FD7F4D12BED690011EE0FD7F4E8056C2
:1020A00090002BE0640260030223AEC3E532955634
:1020B000F534E5319555F533900123E02534FF9053
:1020C0000122E03533FED3EF9400EE94005003027A
:1020D00023AEEF94E8EE940340030223AEE533858C
:1020E00034F012570A900123E0FD7F4912BED690CA
:1020F0000122E0FD7F4A12BED61281C80223AE7BC8
:10210000017A007987E4FD12C10C500EAD177FFFF4
:1021100012BED6AD187FFE02239FE517FE7C00E4B9
:102120002518F532EC3EF53190000BE0FEA3E0FF00
:10213000C3E5329FF534E5319EF53390011FE0256C
:1021400034FF90011EE03533FED3EF9400EE94008F
:1021500050030223AEEF94E8EE940340030223AE53
:10216000E5338534F012570A90011FE0FD7F4D12D0
:10217000BED690011EE0FD7F4E02239F7B017A00B8
:1021800079877D0112C10C500EAD177FFD12BED6AE
:10219000AD187FFC02239FE517FE7C00E42518F5AF
:1021A00032EC3EF53190000DE0FEA3E0FFC3E532D6
:1021B0009FF534E5319EF533900121E02534FF9001
:1021C0000120E03533FED3EF9400EE94005003027B
:1021D00023AEEF94E8EE940340030223AEE533858B
:1021E00034F012570A900121E0FD7F4712BED690CD
:1021F0000120E0FD7F4802239FE517FE7C00E425D7
:1022000018F532EC3EF531900011E0FEA3E0FFC37B
:10221000E5329FF534E5319EF533900125E0253414
:10222000FF900124E03533FED3EF9400EE9400508C
:10223000030223AEEF94E8EE940340030223AEE5DD
:10224000338534F012570A900125E0FD7F4B12BE12
:10225000D6900124E0FD7F4C02239FE517FE7C0011
:10226000E42518F532EC3EF53190000FE0FEA3E0D6
:10227000FFC3E5329FF534E5319EF533900123E04D
:102280002534FF900122E03533FED3EF9400EE9425
:102290000050030223AEEF94E8EE940340030223C0
:1022A000AEE5338534F012570A900123E0FD7F49F3
:1022B00012BED6900122E0FD7F4A02239F7B017A65
:1022C0000079887D0512C10C40030223AEAD177F53
:1022D000FB12BED6AD187FFA02239F7B017A0079EC
:1022E000887D0612C10C40030223AEAD177FF912A0
:1022F000BED6AD187FF802239FAD187FF702239F4B
:10230000900038E0640160030223AEE518B40105D3
:10231000C2440223AEE518640260030223AED24435
:102320000223AEE511640160030223AEAD187F06FF
:1023300012BED690013BE518F07D067CEFE4FF125B
:10234000C0C8806A787AA618E518700890000674EC
:1023500006F0805AE4900006F08053900146800D0C
:1023600090014780089001488003900149E518F0EA
:10237000803C7FF712BE028F35E518700EFB7A00A5
:102380007935E53A24F3FDC261800D7B007A00794E
:1023900035E53A24F3FDD26112BE6EAD357FF712FA
:1023A000BED6800AE5187006C23DF55CF55D900169
:1023B00033E0647F703A753B77AF3B12C122E4F59E
:1023C00035AF357E007B007A00793912ADD8AF3A4F
:1023D00012BE028F36E42535FDE434EEFC12C0C88F
:1023E0000535E535D3941040D8C2AF759F8080FE87
:1023F000900133E0649F7035C2AFC2A9C2AAF59FB5
:1024000075354FAF3512BE028F36E5352402FDE437
:1024100034ECFC12C0C80535E535C394F340E4D272
:0D242000A9D2AAD2AF12C30BE4900133F091
:01242D00228C
:07C2FD00750DFF750AFF2219
:0AC0E80085133F853F99C26AAF3F00
:10C0F200E50A6FFF90664293650DF50AEF9067427D
:03C1020093F50DA5
:01C105002217
:02BF0700A90788
:10BF09007FFF7DFFE4F550AC0119EC601BAE5005D5
:10BF19005074132EF8E66FFC906642936DFF7E0015
:0CBF2900EC90674293FD80DFEFFEEDFF1F
:01BF350022E9
:05B5B30042011A000036
:10B15B00E4900140F0A3F0C2A5C2B4F53ED2B49086
:10B16B000141E025E0FF900140E033FEA2B5E4335E
:10B17B00FDEF4DFFEEF0A3EFF0C2B47F017E0012A6
:10B18B00C251053EE53EC3941040D2D2A5D2B4D2F3
:10B19B00B590014074FF75F0F912570A900140E029
:10B1AB00FEA3E07803CEC313CE13D8F9FF90014072
:10B1BB00EEF0A3EFF07C007D0A12566DA3EEF0A328
:10B1CB00EFF0900142E0C4F854F0C868FEA3E0C46D
:10B1DB00540F48FF900142EEF0A3EFF0900140EEC8
:0CB1EB00F0A3EFF0900140E0FEA3E0FFB5
:01B1F7002235
:1081C80012B15B9000E0EEF0A3EFF0900119E0FF30
:1081D800700690002CE07034EFD3940040069001B4
:1081E80019E014F09000E0E0FEA3E0FF900011EE2B
:1081F800F0A3EFF0EE3395E0FDFCE47B64FAF9F8C8
:108208001257859000F71258210283A8E47B64FA7C
:10821800F9F89000F712580912BC99C39000E1E0F0
:108228009FF53D9000E0E09EF53CC3E53D9428E5D0
:108238003C64809480500CE53D94D8E53C6480947F
:108248007F501D9000F7125815C000AE3CAF3D7C22
:10825800007D0A12566DEE3395E0FDFCD000804992
:10826800D3E53D9400E53C64809480401BD3E53D14
:1082780094FFE53C6480947F500E9000F7125809F3
:10828800E47B01FAF9F88021C3E53D9401E53C64FB
:10829800809480401AE53C6480948050129000F7E6
:1082A80012580974FFFBFAF9F812576A028336E587
:1082B8003D453C7002807D90002CE024FFFFE434B3
:1082C800FFFEE4FCFD9000F7125815125785900048
:1082D800F71258219000F7125815C000C001C002CB
:1082E800C0039000E0E0FEA3E0FFEE3395E0FDFC64
:1082F800E47B64FAF9F8125785D003D002D001D094
:108308000012576A9000F71258219000F712580986
:10831800C004C005C006C00790002CE0FFE4F8F9CF
:10832800FAAB07D007D006D005D00412BC9990004C
:10833800F71258219000F9E0FEA3E0FF7C007D646D
:1083480012567F90013EEEF0A3EFF0C3900012E0CA
:108358009FF53D900011E09EF53CE53DB4FF32E508
:108368003CB4FF2DE47B64FAF9F89000F712580941
:1083780012BC99AC00AD01AE02AF03E47B1EFAF962
:10838800F8D31257E2400A90013E74FFF5F01257F5
:108398000A90013EE0FFA3E0900011CFF0A3EFF0B8
:1083A80090003BE06022900011E0FEA3E0FF7C001B
:1083B8007D0912566D7D051256D4EF2440FFEE3428
:1083C80001900011F0A3EFF0900124E0FEA3E0FF7C
:1083D800900012E02FFF900011E03ECF240CCF3424
:1083E800FEF0A3EFF090002BE0FF700590001180E5
:1083F80010EFB4010590000B8007EF90000FB40256
:1084080009E0F555A3E0F5568019E0FEA3E0FF90DA
:10841800000CE02FFF90000BE03EA2E713F555EFAC
:1084280013F556C3E556940CE5556480947E5006C2
:108438007555FE75560CD3E55694B8E55564809489
:0F8448008B400675550B7556B8E4FDFF02BF6EED
:10C22E009001197405F0E4900099F0FDFF02BF6EC5
:10C1D7009000A1741AF090009A7401F0E4FD7F01B9
